:106DDC000000B30200000301FA0400EF0500030AEF
:106DEC000A5A0B001E0C00FA0D00030E00040F01D2
:106DFC0064100096120132130AFA14010217010AE8
:106E0C001801EF1905321A010A1B01EF1C05321F7C
:106E1C00FFFF20FFFF23011E2400642A00FA2B0031
:106E2C00FA2C50782D003C2E0046300064325078FD
:106E3C003300003432FA35016436016437015038BE
:106E4C000A643A00033B00043C00643E003C3F00F3
:106E5C000040FFFF411450420A5A430AC84405320D
:106E6C004500B44600FA4900024B00014C00FA50B0
:106E7C000404510596520A32530B46540A96570590
:106E8C0046590A465A32FA5B010A5C0A325E000A1B
:106E9C005F00646200FE64FFFF67FFFF6801016929
:106EAC0001016A05966B00006C32966D000473004C
:106EBC00017400017801327901327E006481006432
:106ECC0084FFFF8800028A00019D0A969E00019FA4
:106EDC00FFFFA0FFFFA2000AA3FFFFA4FFFFA5FF77
:106EEC00FFA6FFFFA7FFFFA8FFFFA9FFFF010104FB
:106EFC001501022F003C4701044803045601044EBF
:106F0C00FFFF58000261FFFF6600028500AF86009C
:106F1C00018700FA89010A990008A100FAFAFAFA25
:106F2C000101021501022F1E3C47010448030456BF
:106F3C0001034EFFFF58000261FFFF66000285004F
:106F4C00AF8600018700FA89010A990000A10000B0
:106F5C00FAFAFA0101021501022F1E3C4701024800
:106F6C0003035601014EFFFF58000061FFFF66004E
:106F7C000085FFFF86FFFF87FFFF89010299000054
:106F8C00A10000FAFAFA0065006F00790083008D09
:106F9C00009700A100AC00B600C000CA00D400DE0F
:106FAC0000E800F200580060006800700078008073
:106FBC0000880090009800A000A800B000B800C1A4
:106FCC0000C800D000D800DF00E600EE00F600415B
:106FDC000047004D00530059005F0065006C0071C4
:106FEC000077007D00830089008F0095009B00A234
:106FFC0000A700AC00B200B900C000C500CA00D2A6
:0A700C0000D500DD00E100E700EF11
:103CD80085F97485FA757E017F00E575127128E50E
:103CE800742FFF50010E8E5A8F5B900014E0FCA3D6
:103CF800E0FDEF2DFDEE3CFC8C5C8D5D900034E02A
:103D0800FAA3E0FBED2BFBEC3AFA8A5C8B5D22759B
:103D1800A71085F97485FA757E017F00E575127123
:103D280028E5742FFF50010E8E5A8F5B9000DFE05C
:103D3800B40210AC2DAD2EEF2DFDEE3CFC8C5C8D4D
:103D48005D8016AE5AAF5B900014E0FCA3E0FDEF77
:103D58002DFDEE3CFC8C5C8D5DAE5CAF5D9000345F
:103D6800E0FCA3E0FDEF2DFDEE3CFC8C5C8D5D22BC
:103D7800E55DF5FBE55CF5FCD29322E55DF5E9E54B
:103D88005CF5EAD29422E55DF5EBE55CF5ECD291C1
:103D980022E55DF5EDE55CF5EED2922275A710E51A
:103DA8005DF5FBE55CF5FC75A700D2872275A710C9
:103DB800E55DF5E9E55CF5EA75A700D2902275A7FF
:103DC80010E55DF5EBE55CF5EC75A700E5B544108D
:103DD800F5B52275A710E55DF5EDE55CF5EE75A77F
:103DE80000E5B54420F5B522E50C90698FF8282840
:103DF80073023EB675E700A239B34008E5B544083A
:103E0800F5B58006E5B554F7F5B575E710023EB689
:103E180075E700A239B34008E5B54402F5B5800658
:103E2800E5B554FDF5B575E710023EB6A23992A284
:103E3800807CA23992A1807675E700A239B3400848
:103E4800E5B54440F5B58006E5B554BFF5B575E769
:103E580010805B75E700A239B34008E5B54480F5EA
:103E6800B58006E5B5547FF5B575E7108040A239F1
:103E78009287803AA2399290803475E700A239B3CC
:103E88004008E5B54410F5B58006E5B554EFF5B53D
:103E980075E710801975E700A239B34008E5B54405
:0E3EA80020F5B58006E5B554DFF5B575E710D9
:10698F00023DF9023DFC023E18023E34023E3A023D
:10699F003E40023E5B023E76023E7C023E82023E5B
:0169AF009D4A
:103EB600227434900150F0742B900151F0744890A4
:103EC6000152F0746F900153F0746D900154F074C8
:103ED60065900155F07420900156F07434900157A6
:103EE600F07443900158F07479900159F0746C9015
:103EF600015AF0742090015BF0744490015CF074F8
:103F06007390015DF0747490015EF022900887E072
:103F1600FEA3E0FF741DD39F74019E400C906DDCE0
:103F2600120048E493F599804C90F802E493B405A6
:103F360014900887E0FEA3E0FF906E0F120048E49D
:103F460093F599803090F802E493D3940540149049
:103F56000887E0FEA3E0FF906DDC120048E493F5CD
:103F6600998012900887E0FEA3E0FF906E4212004F
:103F760048E493F599900887127136900887E0FE19
:103F8600A3E0FFEFB45007EEB40103754E0022AE76
:103F96005AAF5B74B48E048F05FF1271188C5C8D5A
:103FA6005DAE5AAF5B74B48E048F05FF1271438CFD
:103FB6005A8D5BC200E55B455A601374B4C3955BCA
:103FC600FFE4955AFE8E5A8F5B785C12717BE5741E
:103FD600A85CB80015D3955D4010E574C3955DFFE8
:103FE600E4955CFE8E5C8F5D8012E5742402C395B9
:103FF6005DFFE4955CFE8E5C8F5DD2002290008DA5
:10400600E0B40104C20A8002D20A90008EE0B40134
:1040160004C20B8002D20B9000CBE075F0D7A4FF50
:10402600AEF0740A8E048F05FF12711890087BECAF
:10403600F0A3EDF09000CBE075F02BA4FFAEF0906E
:104046000010EEF0A3EFF07E017F00900089E012F1
:1040560071289000CCE08E048F05FF127118740A47
:10406600FF1271188D619000D5E075F0D7A4FFAEF0
:10407600F0740A8E048F05FF12711890087FECF019
:10408600A3EDF09000D7E060139000D7E0F5F07450
:104096001684FF7E00EF9008DDF0800674649008B9
:1040A600DDF09000CDE0900066F0900119E0900000
:1040B60073F090011BE0FE9000C9E08E0088F0A42A
:1040C600FFAEF0EF9008E6F09000F4E075F013A470
:1040D600FDACF0900034ECF0A3EDF0A223B3401653
:1040E600900165E0700C900166E07006900167E053
:1040F60060028002C223900165E0B4300F90016631
:10410600E0B44708900167E0643B60028004D22473
:104116008002C22474E3900065F09000B6E0B40B10
:104126000874E3900065F0805A9000B6E0B4191266
:104136009000CCE0906F7D12008CE493900065F0C7
:1041460080419000B6E0B41E129000CCE0906F9BC8
:1041560012008CE493900065F080289000B6E0B4DD
:1041660028129000CCE0906FC512008CE49390006A
:1041760065F0800F9000B6E0B446089000ADE09080
:104186000065F0900086E0FE9008E7E06E601B7523
:1041960099E612019C74AB90003FF012069A746483
:1041A600F5097508001205E480FE90007EE07006B1
:1041B60074009000B3F090006AE0FE9000B3E0B5A2
:1041C600066390006DE0FE9000D1E0B506579000C2
:1041D6006BE0FE9000DFE0B5064B900071E0FE90CC
:1041E6000086E0B5063F90006EE0FE9000C1E0B5A7
:1041F600063390006CE0FE9000CFE0B506279000F5
:104206006FE0FE9000ECE0B5061B900070E0FE90BB
:1042160000EDE0B5060F900072E0FE9000FFE06E44
:10422600700302449C90008EE070089000CFE0641A
:10423600046002800674039000CFF0900047E0C34C
:10424600940550087402900102F080149000DFE09B
:1042560060087406900102F08006740A900102F06C
:10426600900086E0B401067400900086F090008607
:10427600E0B4020674009000D1F0900086E0B4032A
:104286000674009000DEF09000D1E0D39401402740
:10429600741B900104F074009006CFF07400900631
:1042A600D0F0740090009BF09000B3E0B402067466
:1042B600019000B3F080339000B3E0B4021A7400AA
:1042C600900104F074009006CFF074009006D0F0D0
:1042D600741B90009BF080127400900104F0741B14
:1042E6009006CFF0740090009BF09000B3E060144D
:1042F600741C90009AF074009006D3F07400900637
:10430600D4F0800C740090009AF0741C9006D3F0E0
:104316009000ECE060147419900106F074009006A9
:10432600C7F074009006C8F0800C7400900106F087
:1043360074199006C7F09000EDE06014741A9001AD
:1043460007F074009006CBF074009006CCF0800C59
:104356007400900107F0741A9006CBF09000FFE00D
:104366006014742A900777F074009006C3F0740006
:104376009006C4F0800C7400900777F0742A9006BB
:10438600C3F09000DFE0703274059006D7F0740633
:104396009006DBF074079006DFF074089006E3F0F1
:1043A6007400900773F07400900774F0740090071F
:1043B60075F07400900776F0804874009006D7F088
:1043C60074009006D8F074009006DBF07400900636
:1043D600DCF074009006DFF074009006E0F07400E4
:1043E6009006E3F074009006E4F07405900773F00D
:1043F6007406900774F07407900775F074089007B8
:1044060076F09000CFE0D39402401A7415900767B7
:10441600F07416900768F07417900769F074189096
:10442600076AF080277415900767F09000CFE0B414
:1044360002087416900768F080067400900768F00A
:104446007400900769F0740090076AF0D222900019
:10445600B3E090006AF09000DFE090006BF090000F
:10446600D1E090006DF09000C1E090006EF09000F9
:10447600CFE090006CF0900086E0900071F0900024
:10448600ECE090006FF09000EDE0900070F090008E
:10449600FFE0900072F09000E9E0B4011790002070
:1044A600740FF0A374FFF0900022E4F0A3F07402FE
:1044B6009000E9F09000E9E0B40341900022E0FEAC
:1044C600A3E0FF900020E0FCA3E0FD1271737410DE
:1044D6001271287408120039EF9000E8F0EF7006A8
:1044E60074FF9000E8F074009000E9F0900021E07D
:1044F60090009FF0900020E09000A0F090007AE0FD
:10450600900077F0900079E0900076F09000A8E0B7
:10451600C3941E50569000A8E0F404241E90007820
:10452600F0900078E075F0B484FF7E008F74900000
:1045360078E075F0B484ADF07C008D75900076E07F
:10454600D39575400D900076E0C39575900076F092
:10455600800F900076E024B4C39575900076F00540
:1045660074900077E02574900077F0900077E090E3
:10457600003AF090003AE00490003BF090003AE0F8
:10458600D39404400B90003AE0C3940490003AF0B0
:1045960090003BE0D39404400B90003BE0C39404AE
:1045A60090003BF0C22690003AE0D39402400D9072
:1045B600003AE0C3940290003AF0D226C227900057
:1045C6003BE0D39402400D90003BE0C39402900080
:1045D6003BF0D227755E0190007AE0FE9000C0E0C5
:1045E600D39E501390007AE0FE9000C0E0F4042EB3
:1045F6000490003CF0801390007AE02404FE9000C2
:10460600C0E0F4042E0490003CF090003CE0D3940B
:1046160002400F90003CE0C3940290003CF0D21D93
:104626008002C21D90003CE0D39401400B90003CF8
:10463600E01490003DF0800990003CE00490003DBD
:10464600F012019C22C293C294C291C292C287C246
:1046560090E5B554EFF5B5E5B554DFF5B5C296C2AC
:1046660095C2A0C297C2A2C2A1E5B554BFF5B5E5F1
:10467600B5547FF5B5E5B554FBF5B5C20C755F4687
:104686009000C3E07005756E028003756E03755564
:104696000075540090000874FFF0A374DCF0C2119A
:1046A600C21474C8900036F074C8900038F0755380
:1046B60000755200C204754700E570B413037570A7
:1046C60000756400900016E4F0A3F0757110C20F37
:1046D600C210C20375570075560090000AE4F0A395
:1046E600F090000CE4F0A3F0C2297559007558004B
:1046F600900085E075F032A4FFAEF090001EEEF05B
:10470600A3EFF0900074E4F09008E3E4F0C225C251
:104716001AD21BC21CC21DC21E90000EE4F0A3F0EA
:10472600C205C206900074E4F022755B00755A005B
:10473600AE5AAF5B741CC39F74019E50030248249B
:10474600906DDC120048E493645F6023906DDC1288
:104756000048E493647E6017906DDC120048E49391
:104766006481600B906DDC120048E493B48403020C
:104776004804AE5AAF5B906DDC120048E49390009B
:10478600791271590FBF00010EE0FC906DDC12002A
:1047960048ECFEE493FFEEC39F5026AE5AAF5B0F84
:1047A600BF00010E906DDC120048AE5AAF5BE49379
:1047B600FC906DDC120048E493900079127159EC7C
:1047C600F0AE5AAF5B906DDC120048E4939000792E
:1047D600127159E0FC906DDE120048ECFCE493FD8A
:1047E600ECD39D4019906DDE120048E493FC906D69
:1047F600DC120048E493900079127159ECF0AE5A3D
:10480600AF5B74022FFF50010E8E5A8F5B785B747C
:104816000126F6500418E436F640030247362275A0
:104826005B00755A00AE5AAF5B7432BE00039F50F0
:10483600030248F2906EF9120048E4939000791250
:1048460071590FBF00010EE0FC906EF9120048ECA2
:10485600FEE493FFEEC39F5026AE5AAF5B0FBF0038
:10486600010E906EF9120048AE5AAF5BE493FC90CD
:104876006EF9120048E493900079127159ECF0AE8B
:104886005AAF5B906EF9120048E49390007912716A
:1048960059E0FC906EFB120048ECFCE493FDECD36F
:1048A6009D4019906EFB120048E493FC906EF9123D
:1048B6000048E493900079127159ECF0AE5AAF5B60
:1048C600742D6F4E7006755B33755A00AE5AAF5B2A
:1048D60074022FFF50010E8E5A8F5B785B7401268F
:1048E600F6500418E436F6400302482B22755B00A6
:1048F600755A00AE5AAF5B7432BE00039F50030276
:1049060049C0906F2C120048E493900079127159B7
:104916000FBF00010EE0FC906F2C120048ECFEE485
:1049260093FFEEC39F5026AE5AAF5B0FBF00010E3A
:10493600906F2C120048AE5AAF5BE493FC906F2C3C
:10494600120048E493900079127159ECF0AE5AAF18
:104956005B906F2C120048E493900079127159E035
:10496600FC906F2E120048ECFCE493FDECD39D40C6
:1049760019906F2E120048E493FC906F2C12004899
:10498600E493900079127159ECF0AE5AAF5B742D36
:104996006F4E7006755B33755A00AE5AAF5B740284
:1049A6002FFF50010E8E5A8F5B785B740126F650EE
:1049B6000418E436F640030248F922755B00755A7E
:1049C60000AE5AAF5B7432BE00039F5003024A8E9C
:1049D600906F5F120048E4939000791271590FBFEF
:1049E60000010EE0FC906F5F120048ECFEE493FFBE
:1049F600EEC39F5026AE5AAF5B0FBF00010E906FFD
:104A06005F120048AE5AAF5BE493FC906F5F1200F2
:104A160048E493900079127159ECF0AE5AAF5B906E
:104A26006F5F120048E493900079127159E0FC9090
:104A36006F61120048ECFCE493FDECD39D401990A5
:104A46006F61120048E493FC906F5F120048E49394
:104A5600900079127159ECF0AE5AAF5B742D6F4E1F
:104A66007006755B33755A00AE5AAF5B74022FFF42
:104A760050010E8E5A8F5B785B740126F65004182F
:104A8600E436F640030249C72285F97485FA757E35
:104A9600017F00E575127128E5742FFF50010E8E17
:104AA6005A8F5BAC5CAD5DEF2DFDEE3CFC8C5C8DF6
:104AB6005DD293D294D291D292E55DF5FBE55CF599
:104AC600FCE55DF5E9E55CF5EAE55DF5EBE55CF54C
:104AD600ECE55DF5EDE55CF5EE2275A71085F9745C
:104AE60085FA757E017F00E575127128E5742FFF42
:104AF60050010E8E5A8F5B7E017F769000FEE0128B
:104B06007128AC5AAD5BED2FFFEC3EFE8E5C8F5DDF
:104B1600E55DF5FDE55CF5FE900066E4F075A70041
:104B26007412900043F02285F97485FA757E017F30
:104B360000E575127128E5742FFF50010E8E5A8F0D
:104B46005B900010E0FCA3E0FDEF2DFDEE3CFC8C3D
:104B56005C8D5DE55DF5FDE55CF5FE22056522A251
:104B6600D8B34002C293A2D9B34002C294A2DAB328
:104B76004002C291A2DBB34002C292A2DCB3403033
:104B8600A29650067419900043F0A2955006741927
:104B9600900043F0A2A050067419900043F0A2972B
:104BA60050067419900043F0C296C295C2A0C297EF
:104BB60075D8402285A77375A710A2D8B34002C244
:104BC60087A2D9B34002C290A2DAB34006E5B55433
:104BD600EFF5B5A2DBB34006E5B554DFF5B5A2DCCB
:104BE600B340089000CDE0900066F075D84085731C
:104BF600A72290F800E4936406600280FE12009EED
:104C060075A70075D80075D90475DA0975DB0975BD
:104C1600DC0975DD0975DE0975D84075A71075D8EC
:104C26000075D90475DA0975DB0975DC0975DD09C6
:104C360075DE0975D84075A7001200FB74C8F50922
:104C46007508001205E475A70FE5FC900052F0E523
:104C5600FB900053F0E5FA900054F0E5F99000550A
:104C6600F075A70090F800E493F528120703900862
:104C760090E0D394035007900890E0B401067400C6
:104C8600900890F0900890E09008E7F0740190008A
:104C9600C2F0900890E09069B0F8282873802A80C6
:104CA6002875A70F75F30F75A700A2A34006740217
:104CB6009000C2F0801375A70F75F31775A700A2B1
:094CC600A4400674029000C2F043
:0C69B000024CA3024CA5024CA7024CBCF8
:104CCF009000C2E0B4022AC219120AAC740290001A
:104CDF00C2F0900890E09069BCF82828738010808B
:0F4CEF000E74009000D1F0800674009000DEF08B
:0C69BC00024CEC024CEE024CF0024CF8D5
:104CFE008028D2191209C174019000C2F090089058
:104D0E00E09069C8F82828738010800E7400900017
:0A4D1E00D1F0800674009000DEF072
:0C69C800024D16024D18024D1A024D221D
:104D280090F807E49390005FF090005FE0440890EB
:104D3800005FF090005FE054FE90005FF012039D6A
:104D4800123EB790089DE0900165F090089EE090B3
:104D58000166F090089FE0900167F0900165E070AF
:104D68000C900166E07006900167E060028004C262
:104D7800238002D2239000B3E00490006AF0124727
:104D88003090F802E493B405051248F3801290F8C5
:104D980002E493D39405400512482580031249C1C3
:104DA80074009000E9F0124003E5B54401F5B574CC
:104DB80006900045F07400900046F074019000479A
:104DC800F090F802E493900048F090F803E4939090
:104DD8000049F090F804E49390004AF074069000BB
:104DE8004BF0900048E0B40506740590004BF09035
:104DF8000048E0B40406740490004BF07455900029
:104E08004CF0740390004DF0740690004EF0740757
:104E180090004FF090F805E493900050F090F80659
:104E2800E493900051F07400900059F074009000E1
:104E38005AF0740090005BF0740090005CF074000D
:104E480090005DF0740090005EF074FF900060F0D8
:104E5800A2B6B39208A2B3B39209A2A4B39220A2B5
:104E6800A3B39221900061E4F0757000743A900742
:104E780079F074FD90077AF0900062E4F0756F01A4
:104E8800900043E4F09000C3E0B40106741A900067
:104E980043F0C21F756400C20DD20EC203757200C2
:104EA800C222120586756000756C00756200756611
:104EB80032756700756800756900756A00756B0062
:104EC800900016E4F0A3F0756D00D2B2D2A4D2B06F
:104ED800D2B1D2A3D2A7D2A6D2A5D2B77E017F00E3
:104EE8009000A0E012712890009FE02FFF50010E63
:104EF800900020EEF0A3EFF0EFD394FFEE940F4074
:104F080007900020E4F0A3F09000E8E0700674FF3A
:104F18009000E8F09000C3E07005756E028003759C
:104F28006E037400900105F07400900108F074009D
:104F3800900109F074299006BFF0740190076FF092
:104F48007402900770F07403900771F0740490076E
:104F580072F0740090076BF0740090076CF07400A6
:104F680090076DF0740090076EF0D29CE571D394B1
:104F78001040037571109006C0E0D3940C4006747D
:104F8800009006C0F09006C4E0D3940C400674006C
:104F98009006C4F09006C8E0D3940C4006740090C4
:104FA80006C8F09006CCE0D3940C40067400900636
:104FB800CCF09006D0E0D3940C400674009006D054
:104FC800F09006D4E0D3940C400674009006D4F018
:104FD8009006D8E0D3940C400674009006D8F09060
:104FE80006DCE0D3940C400674009006DCF09006D2
:104FF800E0E0D3940C400674009006E0F09006E4DC
:10500800E0D3940C400674009006E4F0D2EC75CF1F
:1050180001A298B34005C298120C14E54E6006A28E
:1050280099B3B340028005C2991210A3E54F6401F9
:105038006005E54FB4040280D5C28E7E087F00E586
:1050480065127128E58D75F008A4FDACF0EF2DFD13
:10505800EE3CFCE58B75F02084FF7E00ED2FFFEC25
:105068003EFE8E548F55D28E9000A6E0605C900074
:1050780018127136900018E0FCA3E0FD90001AE0C9
:10508800FAA3E0FBEDB50342ECB5023EB217A20469
:10509800B3401975E700A217B34008E5B54404F515
:1050A800B58006E5B554FBF5B575E71090001AE034
:1050B800FEA3E0FF90001CE0FCA3E0FDEF2DFDEE59
:1050C8003CFC90001AECF0A3EDF09000B3E060090E
:1050D8009000B3E0C39403400302518F122FCEA275
:1050E80004400890009DE0F546801BE560C395618B
:1050F8005005754600800F90008AE0C395625006FF
:105108009000B0E0F546E54675F002A4FFAEF090D9
:105118000885EEF0A3EFF075E700AC2FAD30EDD3C6
:105128009FEC9E402CE5B5547FF5B59006C0E07025
:1051380006E5B554F7F5B59000B3E0B40209900060
:10514800D1E0C3940240028006E5B54440F5B5803D
:1051580033900061E0C39411502AE5B54480F5B559
:105168009006C0E07006E5B54408F5B59000B3E0D8
:10517800B402099000D1E0C3940240028006E5B56C
:1051880054BFF5B575E7109000B3E0B4032A1230A8
:10519800E975E700AE2FAF30900885E0FCA3E0FD8D
:1051A800EFD39DEE9C4008E5B54480F5B58006E553
:1051B800B5547FF5B575E710A2B3300901B340596E
:1051C800A2B3300901B34051A2B3300B01B3403C44
:1051D800A20CB340329000C1E0B40406A21AB3B3E3
:1051E800400280067405900043F0D21AD205C20628
:1051F800E55F64026005E55FB40402800AE56E704D
:10520800067403900043F0A20BB39209A20BB330CB
:10521800B301B34004A20B9209A2B6300801B350FF
:10522800030257D5A2B6300801B350030257D5A2DE
:10523800B6300A01B35003025707756F00055FA225
:1052480005B35003025348E56EB4034EA229B34098
:1052580042E55FB40503756E01A206401CE55FC315
:10526800940350069000437401F0E55FD394034023
:10527800067402900043F0801AE55FC39405500657
:105288009000437401F0E55FD394054006740290E2
:105298000043F0755F01D229805EE56EB4020675A1
:1052A8006E01755F03E55FB40305755F0180499082
:1052B8000043E07034E55FC39403500690004374E4
:1052C80001F0E55FD3940340067402900043F0E5D3
:1052D8005FC394035002D21FE55FD394034002D208
:1052E8001FC296C295C2A0C2979000C3E0B4010540
:1052F80012464B8003755F01C20574029008E3F003
:10530800A21FB34002C21FA21AB34006A21D921CDC
:105318008002B21CD21BE56E700EA21AB35009A20D
:105328001C301D01B3B3400280067405900043F0A1
:10533800C21AA2A4B34002C220A2A3B34002C2214F
:10534800E56EC394035006E55F640360028045A2DE
:105358001AB34006A21D921C8002B21CE56E700EA4
:10536800A21AB35009A21C301D01B3B34002800633
:105378007405900043F0C21AC21B755F01D206A2E1
:10538800A4B34002C220A2A3B34002C221A21FB309
:105398004002C21FA206B3B35006E55F6403600271
:1053A80080127405900043F0D21F9000C3E0B4014E
:1053B8000312464BE55FB4024F9000A6E0604990A7
:1053C8000018E0FEA3E0FF9000A6E08E048F05FF22
:1053D80012711874018C068D0712003990001CEEAA
:1053E800F0A3EFF090001CE0F8A3E090001AC8F0DA
:1053F800A3C8F0900018E4F0A3F0C21775E700E521
:10540800B554FBF5B575E710AE58AF59AC54AD556A
:10541800EF2DFDEE3CFC8C588D59AE54AF55EFD3B3
:105428009DEE9C401190000EE0FAA3E0FBEBC394C4
:10543800E8EA94034002800690000E12713690004C
:1054480008E554F0A3E555F090000AE554F0A3E50B
:1054580055F0AE54AF5574128E048F05FF127118B3
:105468008C568D57C28E758D00758B0075650075CD
:105478005501755400D28E900008E0FEA3E0FFEFBE
:105488004E600B7C7E7D781270168E528F53AE5212
:10549800AF537428BE00039F5010E5642FFF5001DE
:1054A8000E74011200398E528F538553649000CACE
:1054B800E0A852B8000DD395534008E55390004238
:1054C800F080099000CAE014900042F0E56E600692
:1054D8007553007552009000C1E0B4040890003C78
:1054E800E0655F6002800BA21CB34004D21E8002FC
:1054F800B21E9000B3E06003122C84E570B413036D
:10550800757000A20D500302567E9000CFE0C39440
:10551800045006A20CB3B340030255C990007FE0C3
:10552800B40173900101E0B40214121244900067B0
:10553800E075F0BCA4FFAEF08E5C8F5D8056E56828
:1055480075F00A84FF7E00900579120048E0F55B4B
:10555800755A00AE5AAF5B9000A4E01271287464CB
:105568008E048F05FF1271188C5C8D5DE55D9000CF
:105578003EF0AE5AAF5B90007DE012712874648EE5
:10558800048F05FF12711874BC8C068D07127128E0
:105598008E5C8F5D801790007DE075F0BCA4FFAE37
:1055A800F08E5C8F5D9000A4E090003EF0E562C351
:1055B80094CC5006E55D455C70028003124A8FD298
:1055C8000D9000CFE0B404069008E3E070030256A3
:1055D8007E90007FE0B40173900101E0B4021412E0
:1055E8001244900067E075F0BCA4FFAEF08E5C8FAB
:1055F8005D8056E56875F00A84FF7E009005791293
:105608000048E0F55B755A00AE5AAF5B9000A4E025
:1056180012712874648E048F05FF1271188C5C8DCA
:105628005DE55D90003EF0AE5AAF5B90007DE01204
:10563800712874648E048F05FF12711874BC8C066F
:105648008D071271288E5C8F5D801790007DE07544
:10565800F0BCA4FFAEF08E5C8F5D9000A4E09000DB
:105668003EF0E562C394CC5006E55D455C7002806F
:1056780003124A8FD20DE56EB40106A20CB3B340F3
:105688000280189000CFE0B4040575710380097595
:1056980071009000447401F0756E00E56E705B90C7
:1056A80000C6E0600D900066E0A852B80006955369
:1056B800400280299000C6E0B40208757103756D38
:1056C80000800CC201756D00900016E4F0A3F09004
:1056D8000066E060067409900043F0801D75710053
:1056E80090003AE0B55F069000447401F090003BEA
:1056F800E0B55F067402900044F0A20AB39208A2D3
:105708000AB330B601B350030257D5756F0175E778
:1057180000E5B54401F5B575E710740B900061F02C
:10572800A20A9208E55FD394474014D20CE55FD3F0
:10573800944B400B7405900043F0D21F755F469060
:1057480000CEE0B40107E56BC3944140028018E540
:105758006BC3941450087413900043F08006740EC1
:10576800900043F012464B90004BE0FE900048E05A
:10577800C39E4009900048E0D39408400974FB9008
:105788000043F012464B900049E06015900049E054
:10579800FE900047E06E600974FC900043F01246EA
:1057A8004B90004AE0601590004AE0FE90004CE003
:1057B8006E600974FE900043F012464B900890E02A
:1057C80060069000FEE060028003120B97A21FB3F0
:1057D8004008C296C295C2A0C2979000FEE0600C35
:1057E800AE52AF537414BE00059F4002803790003C
:1057F80086E09069D4F8282873802A8028A2A3B369
:105808005005A221B340028005124AE0D22180153A
:10581800A2A4B35005A220B340028005124AE0D2E8
:05582800208002800059
:1069D40002580102580302580502581802582B02A3
:0269E400582D2C
:10582D00A20FB3B3500890003CE0655F6003025BCC
:10583D0028A202B35006A201B3B34003025B249029
:10584D0000C1E0B404028003025B009008E3E0B401
:10585D0002028003025AF5A21EB350030259AE1282
:10586D003CD8900112E0601F900014E0FEA3E0FF11
:10587D0090010AE012712874C88E048F05FF127111
:10588D00188C5C8D5D800A900014E0F55CA3E0F54A
:10589D005DAE5CAF5D745E12712874058E048F056C
:1058AD00FF127118AE5AAF5BED2FFFEC3EFE8E5C12
:1058BD008F5D900034E0FCA3E0FDEF2DFDEE3CFC90
:1058CD008C5C8D5D123D78A203B34068123D17903C
:1058DD000112E0601F900014E0FEA3E0FF90010AAA
:1058ED00E012712874C88E048F05FF1271188C5C3C
:1058FD008D5D800A900014E0F55CA3E0F55DAE5C73
:10590D00AF5D745E12712874058E048F05FF1271E0
:10591D0018AE5AAF5BED2FFFEC3EFE8E5C8F5D90A7
:10592D000034E0FCA3E0FDEF2DFDEE3CFC8C5C8D26
:10593D005D123DA49000DFE0B40263123D179001AB
:10594D0012E0D39404401BAE2DAF2E90010EE01249
:10595D00712874C88E048F05FF1271188C5C8D5DD3
:10596D008006852D5C852E5DAE5CAF5D745E12711B
:10597D002874058E048F05FF127118AE5AAF5BEDBA
:10598D002FFFEC3EFE8E5C8F5D900034E0FCA3E0BB
:10599D00FDEF2DFDEE3CFC8C5C8D5D123DA4025A9D
:1059AD00F3123CD8900112E0D39403401F900014E1
:1059BD00E0FEA3E0FF90010CE012712874C88E0484
:1059CD008F05FF1271188C5C8D5D800A900014E0BC
:1059DD00F55CA3E0F55DAE5CAF5D745E127128748D
:1059ED00058E048F05FF127118AE5AAF5BED2FFFB8
:1059FD00EC3EFE8E5C8F5D900034E0FCA3E0FDEF8D
:105A0D002DFDEE3CFC8C5C8D5D123D8EA203B340F2
:105A1D006B123D17900112E0D39403401F900014B8
:105A2D00E0FEA3E0FF90010CE012712874C88E0413
:105A3D008F05FF1271188C5C8D5D800A900014E04B
:105A4D00F55CA3E0F55DAE5CAF5D745E127128741C
:105A5D00058E048F05FF127118AE5AAF5BED2FFF47
:105A6D00EC3EFE8E5C8F5D900034E0FCA3E0FDEF1C
:105A7D002DFDEE3CFC8C5C8D5D123DC69000DFE093
:105A8D00B40263123D17900112E0D39406401BAE91
:105A9D002DAF2E900110E012712874C88E048F0561
:105AAD00FF1271188C5C8D5D8006852D5C852E5DD9
:105ABD00AE5CAF5D745E12712874058E048F05FFA8
:105ACD00127118AE5AAF5BED2FFFEC3EFE8E5C8F60
:105ADD005D900034E0FCA3E0FDEF2DFDEE3CFC8C71
:105AED005C8D5D123DC68009123CD8123D78123D89
:105AFD008E8024123CD8123D78123D8EA203B34005
:105B0D0006123DA4123DC69000DFE0B40209123D1D
:105B1D0017123DA4123DC6C20FD210A210B3B3503E
:105B2D000890003DE0655F6003025E29A202B3505C
:105B3D0006A201B3B34003025E259000C1E0B40498
:105B4D00028003025E019008E3E0B40202800302CA
:105B5D005DF6A21EB35003025CAF123CD890011249
:105B6D00E0D39401401F900014E0FEA3E0FF9001EC
:105B7D000BE012712874C88E048F05FF1271188CFA
:105B8D005C8D5D800A900014E0F55CA3E0F55DAEE0
:105B9D005CAF5D745E12712874058E048F05FF1263
:105BAD007118AE5AAF5BED2FFFEC3EFE8E5C8F5D34
:105BBD00900034E0FCA3E0FDEF2DFDEE3CFC8C5C91
:105BCD008D5D123D83A203B3406B123D1790011200
:105BDD00E0D39401401F900014E0FEA3E0FF90017C
:105BED000BE012712874C88E048F05FF1271188C8A
:105BFD005C8D5D800A900014E0F55CA3E0F55DAE70
:105C0D005CAF5D745E12712874058E048F05FF12F2
:105C1D007118AE5AAF5BED2FFFEC3EFE8E5C8F5DC3
:105C2D00900034E0FCA3E0FDEF2DFDEE3CFC8C5C20
:105C3D008D5D123DB59000DFE0B40263123D17900B
:105C4D000112E0D39405401BAE2DAF2E90010FE055
:105C5D0012712874C88E048F05FF1271188C5C8D1B
:105C6D005D8006852D5C852E5DAE5CAF5D745E122C
:105C7D00712874058E048F05FF127118AE5AAF5B33
:105C8D00ED2FFFEC3EFE8E5C8F5D900034E0FCA3AB
:105C9D00E0FDEF2DFDEE3CFC8C5C8D5D123DB50203
:105CAD005DF4123CD8900112E0D39403401F900094
:105CBD0014E0FEA3E0FF90010DE012712874C88E70
:105CCD00048F05FF1271188C5C8D5D800A90001495
:105CDD00E0F55CA3E0F55DAE5CAF5D745E1271281E
:105CED0074058E048F05FF127118AE5AAF5BED2F40
:105CFD00FFEC3EFE8E5C8F5D900034E0FCA3E0FD7A
:105D0D00EF2DFDEE3CFC8C5C8D5D123D99A203B335
:105D1D00406B123D17900112E0D39403401F900089
:105D2D0014E0FEA3E0FF90010DE012712874C88EFF
:105D3D00048F05FF1271188C5C8D5D800A90001424
:105D4D00E0F55CA3E0F55DAE5CAF5D745E127128AD
:105D5D0074058E048F05FF127118AE5AAF5BED2FCF
:105D6D00FFEC3EFE8E5C8F5D900034E0FCA3E0FD09
:105D7D00EF2DFDEE3CFC8C5C8D5D123DDB9000DF6C
:105D8D00E0B40263123D17900112E0D39407401B5B
:105D9D00AE2DAF2E900111E012712874C88E048FB4
:105DAD0005FF1271188C5C8D5D8006852D5C852E2E
:105DBD005DAE5CAF5D745E12712874058E048F0547
:105DCD00FF127118AE5AAF5BED2FFFEC3EFE8E5CED
:105DDD008F5D900034E0FCA3E0FDEF2DFDEE3CFC6B
:105DED008C5C8D5D123DDB8009123CD8123D831217
:105DFD003D998024123CD8123D83123D99A203B3E4
:105E0D004006123DB5123DDB9000DFE0B4020912F1
:105E1D003D17123DB5123DDBD20FC210E5719069F1
:095E2D00E6F82828739000E6E075
:0369E600025E321C
:105E3600906A55F82828731225CF80121225CF8034
:0E5E46000D1226598008122705800312270529
:0F6A5500025E3D025E42025E47025E4C025E51EF
:105E540075710102622212283112294875710202F9
:105E64006222122CC8A204B340139000CBE075F058
:105E74001DA4FFAEF0900010EEF0A3EFF0900879AF
:105E8400E0FEA3E0FF740A12712890000AE0FCA36C
:105E9400E0FD74098F02FF1271188D078C038E04C4
:105EA4008A058B0612701690087DEEF0A3EFF09031
:105EB40000CFE0B401087478BE00059F4002800D55
:105EC400747890087DF8E4F0E8A3F0801B90087DD6
:105ED400E0FEA3E0FF74F0BE00039F500B74F0904B
:105EE400087DF8E4F0E8A3F0E53770037537019016
:105EF400087DE0FEA3E0FFE5372FFF50010E900878
:105F04007DEEF0A3EFF0757103A2304015900044CC
:015F1400E0AC
:0669E900025E5A025E6628
:105F1500906A64F8282873800875710A8003757182
:015F25000B70
:096A6400025F1C025F1E025F23A9
:105F26000262229006C0E060077401F508122DF6A1
:105F3600A232B3401675E700900777E0B42A06E56B
:105F4600B54402F5B575E710025FF29000B4E0D3F0
:105F560094024045900088E02403A852B8000495B6
:105F660053500990008AE0D395625002800ED20207
:105F7600A22840067408900043F0D228900088E0DA
:105F8600A852B80005D39553500B90008AE024031D
:105F9600C395625002C2028053900088E02403A891
:105FA60052B8000495535010E560C39561500990AE
:105FB600008AE0D395625002800ED202A2284006E3
:105FC6007408900043F0D228900088E0A852B800E8
:105FD60005D395535014E561240FC39560400B908B
:105FE600008AE02403C395625002C202A202400264
:105FF600C2289000FFE0B4010AA232B35005A20203
:10600600B34002801375E700900777E0B42A06E5EF
:10601600B554FDF5B575E7109000CEE07007E56B59
:10602600C3941440028002D2029000C3E0B401027D
:10603600D202A2024005757104800A7571109000A3
:0C60460016E4F0A3F00262229000B4E027
:0669EF00025F2902604E68
:10605200906A6DF828287312135A801212135A800C
:0E6062000D12150D80081215C480031215C40E
:0F6A6D0002605902605E02606302606802606D41
:106070009006C4E060077402F508122DF6757105EC
:1060800002622212171D7571069006C8E06007743F
:1060900003F508122DF69006CCE060077404F508AD
:1060A000122DF602622290003EE06006A204B3B315
:1060B0004002800DE55FD39401500690003EE0144D
:1060C000F01219A67571079006D0E060077405F507
:1060D00008122DF69006D4E060077406F508122D1C
:1060E000F6026222900101E0B402031212CB121EEA
:1060F0000E7571089006D8E060077407F508122D38
:10610000F69006DCE060077408F508122DF60262CE
:1061100022121EF07571090262221222C8A20FB368
:106120005005A210B340028004D20FD21075711036
:106130009006E0E060077409F508122DF69006E479
:10614000E06007740AF508122DF60262229000370B
:10615000E0C39446500AC296C2A07446900037F03D
:1061600085375B755A0090003AE0F574123F95E56B
:106170005D900037F0900004E55AF0A3E55BF0C2B3
:106180001290087DE0F55AA3E0F55B90003AE0F547
:1061900074123F95E55D900036F0900000E55AF0EE
:1061A000A3E55BF0A2009213C21175710380739096
:1061B0000039E0C3944650139000CFE0B40102C20E
:1061C00096C295C2977446900039F085375B755A30
:1061D0000090003BE0F574123F95E55D900039F0CA
:1061E000900006E55AF0A3E55BF0C21590087DE04B
:1061F000F55AA3E0F55B90003BE0F574123F95E59E
:106200005D900038F0900002E55AF0A3E55BF0A243
:10621000009216C214757103800880068004800203
:026220008000FC
:1069F5000260830260A60260E402611102611A026C
:106A0500614D0261AF02621A02621C02621E0262DD
:046A150020026222D7
:10622200900036E0B55F0280030262F8A211406B73
:10623200900000E0FEA3E0FFEF4E605DAC52AD5374
:10624200740ABC0033D39D402FAA56AB5774058AFB
:10625200048B05FF1271188D068C07900000E0FC7C
:10626200A3E0FDCFCECF12000374011200399000DB
:1062720000EEF0A3EFF08021AE56AF57900000E0A1
:10628200FCA3E0FD120003740A8E048F05FF127155
:1062920018900000ECF0A3EDF0D211AE54AF55907F
:1062A2000000E0FCA3E0FDEFC39DEE9C4048124BD2
:1062B2002D9000CFE0906A19F82828738030D2968A
:1062C200802CD2968028D296D2A08022A21340108F
:1062D200A226301B01B34004D2A08002D296800EC7
:0E62E200A226301B01B34004D2968002D2A047
:0F6A19000262BE0262C00262C40262C80262CEA2
:1062F000C21174C8900036F0A211B3B350079000D9
:1063000036E0B55F028048124B2D9000CFE0906AD6
:1063100028F82828738030D296802CD2968028D2F4
:1063200096D2A08022A2134010A226301B01B340B7
:1063300004D2A08002D296800EA226301B01B34068
:0763400004D2968002D2A0F6
:0F6A280002631502631702631B02631F026325DB
:1063470074C8900036F0C211900037E0B55F028044
:10635700030263E9A212406B900004E0FEA3E0FF92
:10636700EF4E605DAC52AD53740ABC0033D39D4011
:106377002FAA56AB5774058A048B05FF1271188D27
:10638700068C07900004E0FCA3E0FDCFCECF1200FF
:10639700037401120039900004EEF0A3EFF080219E
:1063A700AE56AF57900004E0FCA3E0FD1200037463
:1063B7000A8E048F05FF127118900004ECF0A3ED0C
:1063C700F0D212AE54AF55900004E0FCA3E0FDEF0D
:1063D700C39DEE9C400CC296C2A07446900037F055
:1063E700C212A212B3B35007900037E0B55F028024
:1063F7000CC296C2A07446900037F0C212900038C3
:10640700E0B55F0280030264DAA214406B900002D9
:10641700E0FEA3E0FFEF4E605DAC52AD53740ABCE3
:106427000033D39D402FAA56AB5774058A048B05BA
:10643700FF1271188D068C07900002E0FCA3E0FDA7
:10644700CFCECF1200037401120039900002EEF094
:10645700A3EFF08021AE56AF57900002E0FCA3E017
:10646700FD120003740A8E048F05FF127118900045
:1064770002ECF0A3EDF0D214AE54AF55900002E059
:10648700FCA3E0FDEFC39DEE9C4048124B2D90000E
:10649700CFE0906A37F82828738030D296802CD2C4
:1064A700958028D295D2978022A2164010A2273035
:1064B7001B01B34004D2978002D295800EA22730E9
:0B64C7001B01B34004D2958002D29765
:0F6A37000264A00264A20264A60264AA0264B010
:1064D200C21474C8900038F0A214B3B350079000ED
:1064E20038E0B55F028048124B2D9000CFE0906AF1
:1064F20046F82828738030D296802CD2958028D2F4
:1065020095D2978022A2164010A227301B01B340D9
:1065120004D2978002D295800EA227301B01B3408D
:0765220004D2958002D2971C
:0F6A46000264F70264F90264FD0265010265074C
:1065290074C8900038F0C214900039E0B55F028059
:10653900030265D4A215406B900006E0FEA3E0FFBC
:10654900EF4E605DAC52AD53740ABC0033D39D402D
:106559002FAA56AB5774058A048B05FF1271188D43
:10656900068C07900006E0FCA3E0FDCFCECF120019
:10657900037401120039900006EEF0A3EFF08021B8
:10658900AE56AF57900006E0FCA3E0FD120003747D
:106599000A8E048F05FF127118900006ECF0A3ED26
:1065A900F0D215AE54AF55900006E0FCA3E0FDEF24
:1065B900C39DEE9C40159000CFE0B40102C296C283
:1065C90095C2977446900039F0C215A215B3B3501D
:1065D90007900039E0B55F0280159000CFE0B40163
:1065E90002C296C295C2977446900039F0C21590BE
:1065F90000D1E0B40202800302672C900063E0D36B
:1066090095675064900063E0F4042567FE9000D418
:10661900E08E00F5F0E884FF7E008F74EFC39410DC
:10662900500CEF8574F0A4FDACF08D748003757483
:10663900FF900063E0D39574400B900063E0C3952D
:1066490074F57280037572009000EFE0D395724083
:10665900069000EFE0F5729000F0E0C395725006E5
:106669009000F0E0F5728071900063E0C39567FED9
:106679009000D4E08E00F5F0E884FF7E008F74EF7F
:10668900C39410500CEF8574F0A4FDACF08D7480A8
:10669900037574FF85745B755A00900063E0255B90
:1066A900FFAE5A50010E8E5A8F5B74FFBE0009D39C
:1066B9009F4005855B7280037572FF9000EFE0D300
:1066C900957240069000EFE0F5729000F0E0C395F6
:1066D9007250069000F0E0F572A204B3B3500D9029
:1066E9000064E0FE9000DCE0D39E50028014740741
:1066F900900043F075E700E5B554BFF5B575E710AF
:10670900802175A71075E700E5CDC395724008E5AE
:10671900B554BFF5B58006E5B54440F5B575E71044
:1067290075A7009000ECE0604E9000F6E0A852B822
:106739000004955350179000F5E0A852B8000ED305
:10674900955340099000F7E0D39562400280157592
:10675900A710E5CDC394BF4004C2A28002D2A2759E
:10676900A700801375A710E5CDC394404004C2A2C9
:106779008002D2A275A7009000EDE0604E9000F96A
:10678900E0A852B80004955350179000F8E0A852B9
:10679900B8000ED3955340099000FAE0D3956240B2
:1067A90002801575A710E5CDC394BF4004C2A1802E
:1067B90002D2A175A700801375A710E5CDC3944037
:1067C9004004C2A18002D2A175A700E570C3941349
:1067D900501DE57075F00284AFF07E00EF4E700534
:1067E900123290800AA2EDB34005C2ED123290AE8A
:1067F90054AF5574B8C39F74889E400C900062E0F2
:10680900C3945A400302698CA20CB3400912464B47
:106819007406900043F0A20EB3500EE562D3943390
:106829004007E562C394CC40028041900101E0B485
:106839000214121244900067E075F05EA4FFAEF0F6
:106849008E5C8F5D800F90007DE075F05EA4FFAED9
:10685900F08E5C8F5DE55D455C6011E5B54401F541
:10686900B5740B900061F0124A8FD20E900062E06D
:10687900D394014007E562C3941A40028002C20E14
:106889009006C0E060077401F508122DF69006C461
:10689900E060077402F508122DF69006C8E060075B
:1068A9007403F508122DF69006CCE060077404F520
:1068B90008122DF69006D0E060077405F508122D30
:1068C900F69006D4E060077406F508122DF69006D6
:1068D900D8E060077407F508122DF69006DCE06031
:1068E900077408F508122DF69006E0E060077409B0
:1068F900F508122DF69006E4E06007740AF508120F
:106909002DF6900062E0C3945A5010E570B4130953
:10691900900062E004F0757000803FE570B41303E5
:10692900757000C28E758D00758B00756500755583
:1069390001755400D28E900061E0C3941150089003
:106949000061E004F080067411900061F09000612C
:10695900E0B41106E5B554FEF5B5900062E0D394B4
:10696900014007E56BC3944140028006740E900014
:1069790043F0900890E060069000FEE0600280031A
:06698900120B97025016EC
:106A7C000000010001400160018001A001C001E0A3
:106A8C0002000300039603B603D603F404000500CA
:106A9C000512052405360548055A056C057E05903A
:106AAC0005A805C005DE0600061406280646066E77
:106ABC0006AE05CF06EE00FF013F015F017F019F8F
:106ACC0001BF01DF01FF02FF039503B503D503F3FB
:106ADC0003FF04FF05110523053505470559056B13
:106AEC00057D058F05A705BF05CE05F10613062705
:106AFC000645066D06AD06ED05DD06FF0FAA0FA5D2
:106B0C000F9F0F9A0F940F8D0F870F800F780F71B7
:106B1C000F680F600F570F4E0F450F3B0F300F25AF
:106B2C000F1A0F0E0F020EF50EE80EDB0ECC0EBE7A
:106B3C000EAE0E9F0E8E0E7D0E6C0E5A0E470E3440
:106B4C000E200E0C0DF70DE20DCB0DB50D9D0D8528
:106B5C000D6D0D540D3A0D200D050CE90CCE0CB13C
:106B6C000C940C760C580C3A0C1B0BFB0BDB0BBB74
:106B7C000B9A0B790B570B350B130AF10ACE0AAB98
:106B8C000A870A640A400A1C09F809D409B0098C5E
:106B9C0009670943091F08FB08D608B2088E086A62
:106BAC000846082307FF07DC07B907960773075148
:106BBC00072F070D06EC06CA06AA068906690649C0
:106BCC00062A060A05EC05CD05B005920575055893
:106BDC00053C0520050504EA04CF04B5049C048299
:106BEC000469045104390422040B03F403DE03C8C2
:106BFC0003B2039D038903750361034D033B032813
:106C0C000316030402F202E102D102C002B002A098
:106C1C00029102820273026502570249023C022F62
:106C2C0002220216020901FD01F201E601DB01D08C
:106C3C0001C601BB01B101A7019D0194018B018229
:106C4C00017901700168016001580150014801414E
:106C5C0001390132012B0125011E01180111010B13
:106C6C00010500FF00FA0FA60FA00F990F920F8BD2
:106C7C000F840F7C0F740F6B0F620F580F4E0F4366
:106C8C000F380F2C0F1F0F120F050EF70EE80ED832
:106C9C000EC80EB70EA50E930E800E6C0E580E423B
:106CAC000E2C0E150DFD0DE40DCB0DB10D950D79C2
:106CBC000D5D0D3F0D200D010CE10CC00C9E0C7CEC
:106CCC000C590C350C100BEA0BC40B9E0B760B4FAE
:106CDC000B260AFD0AD40AAA0A800A550A2A09FFB9
:106CEC0009D409A8097C0950092508F908CD08A17F
:106CFC000875084A081E07F307C8079D077307495C
:106D0C00072006F706CE06A6067E06570630060AAC
:106D1C0005E405BF059B057705540532051004EF06
:106D2C0004CE04AE048F047104530435041903FD1E
:106D3C0003E203C703AD0394037B0363034B0334E8
:106D4C00031E030802F302DE02CA02B602A302917A
:106D5C00027F026D025C024C023C022C021D020EF0
:106D6C00020001F201E401D701CA01BE01B101A682
:106D7C00019A018F0185017A01700166015D015351
:106D8C00014A014101390131012901210119011285
:106D9C00010B010400FD00F700F000EA00E400DE46
:106DAC0000D900D300CE00C900C400BF00BA00B5A2
:106DBC0000B100AD00A800A400A0009C00990095B3
:106DCC000091008E008A008700840081007E007B89
:10009E0075B50075840175A70075FFA075EF069004
:1000AE00003FE4F075C91075A70F75A1C775A700BD
:1000BE0075D90075CE0C75A70F75F1FE75F2FF752B
:1000CE00F30775F47875A4BA75A5FF75A60775AE16
:1000DE000075AFFF75D48175D5FF75D6FF75D7FF47
:1000EE0075A70075A20175A14775F8092275E60876
:1000FE0075E71075BC0175BE0475BD6C75BE0775D0
:10010E00BDA075BE0875BD0175BC0075BB1875BC6C
:10011E002075BA0875E88075D11375A70F75E105BE
:10012E0075E20075C74012464B759700759780743F
:10013E000A1271087597C0E5975420700280F87501
:10014E008F0275A700D2AF75980075A90C75A70F11
:10015E0075AB4375ADFB75AC1E75A71075C91875DB
:10016E00CA0075CB0075C80475A700758912758E07
:10017E0004758C00758A00C2A9D28C758D00758BA2
:10018E0000D2ABD28E75B62075D944C2992290009A
:10019E007BE090088FF0900086E0900890F0900041
:1001AE0087E0900891F09000A6E0900892F0900001
:1001BE00B3E0900893F09000C1E0900894F09000A6
:1001CE00CFE0900895F09000D1E0900896F0900066
:1001DE00DFE0900897F09000ECE0900898F0900027
:1001EE00EDE0900899F09000FFE090089AF09001F1
:1001FE0017E090089CF0900165E090089DF090014A
:10020E0066E090089EF0900167E090089FF09000E5
:10021E00FEE09008A0F09000E8E09008A1F09000B9
:10022E009FE09008A2F09000A0E09008A3F090004C
:10023E009AE09008A4F090009BE09008A5F0900141
:10024E0004E09008A6F0900105E09008A7F0900158
:10025E0006E09008A8F0900107E09008A9F0900140
:10026E0008E09008AAF09006BFE09008ABF0900668
:10027E00C3E09008ACF09006C7E09008ADF0900691
:10028E00CBE09008AEF09006CFE09008AFF090066D
:10029E00D3E09008B0F09006D7E09008B1F0900649
:1002AE00DBE09008B2F09006DFE09008B3F0900625
:1002BE00E3E09008B4F0900767E09008B5F090077F
:1002CE0068E09008B6F0900769E09008B7F09007E4
:1002DE006AE09008B8F090076BE09008B9F09007CC
:1002EE006CE09008BAF090076DE09008BBF09007B4
:1002FE006EE09008BCF090076FE09008BDF090079C
:10030E0070E09008BEF0900771E09008BFF0900783
:10031E0072E09008C0F0900773E09008C1F090076B
:10032E0074E09008C2F0900775E09008C3F0900753
:10033E0076E09008C4F0900777E09008C5F0900141
:10034E0009E09008C6F090010AE09008C7F090010D
:10035E000BE09008C8F090010CE09008C9F09001F5
:10036E000DE09008CAF090010EE09008CBF09001DD
:10037E000FE09008CCF0900110E09008CDF09001C5
:10038E0011E09008CEF0900112E09008CFF022908C
:10039E00088FE090007BF0900890E0900086F0903F
:1003AE000891E0900087F0900892E09000A6F090FF
:1003BE000893E09000B3F0900894E09000C1F090A4
:1003CE000895E09000CFF0900896E09000D1F09064
:1003DE000897E09000DFF0900898E09000ECF09025
:1003EE000899E09000EDF090089AE09000FFF090F0
:1003FE00089CE0900117F09008A0E09000FEF090AD
:10040E0008A1E09000E8F09008A2E090009FF09024
:10041E0008A3E09000A0F09008A4E090009AF0905D
:10042E0008A5E090009BF09008A6E0900104F090E3
:10043E0008A7E0900105F09008A8E0900106F09062
:10044E0008A9E0900107F09008AAE0900108F0904A
:10045E0008ABE09006BFF09008ACE09006C3F090B9
:10046E0008ADE09006C7F09008AEE09006CBF09095
:10047E0008AFE09006CFF09008B0E09006D3F09071
:10048E0008B1E09006D7F09008B2E09006DBF0904D
:10049E0008B3E09006DFF09008B4E09006E3F09029
:1004AE0008B5E0900767F09008B6E0900768F09006
:1004BE0008B7E0900769F09008B8E090076AF090EE
:1004CE0008B9E090076BF09008BAE090076CF090D6
:1004DE0008BBE090076DF09008BCE090076EF090BE
:1004EE0008BDE090076FF09008BEE0900770F090A6
:1004FE0008BFE0900771F09008C0E0900772F0908E
:10050E0008C1E0900773F09008C2E0900774F09075
:10051E0008C3E0900775F09008C4E0900776F0905D
:10052E0008C5E0900777F09008C6E0900109F090BA
:10053E0008C7E090010AF09008C8E090010BF09017
:10054E0008C9E090010CF09008CAE090010DF090FF
:10055E0008CBE090010EF09008CCE090010FF090E7
:10056E0008CDE0900110F09008CEE0900111F090CF
:10057E0008CFE0900112F022754800900887E4F051
:10058E00A3F0753200753100754E00754F00C22C08
:10059E00D22D900890E06002D22274FE900889F865
:1005AE00E4F0E8A3F074FE90088DF8E4F0E8A3F010
:1005BE0074FE90088BF8E4F0E8A3F0745A9008E10A
:1005CE00F0745A9008E2F0D22EC22AC230C22FC264
:1005DE002BC232C23822750B00750A00AE0AAF0B61
:1005EE00AC08AD09EDC39FEC9E401674FF12710866
:1005FE0075CF01780B740126F6500418E436F650C8
:10060E00DB22C2AF75D904758F0375B7A575B7F127
:10061E0090F800E4F0758F0175B7A575B7F1E52870
:10062E0090F800F075B7A575B7F190F801E4F07584
:10063E00B7A575B7F19008D5E090F802F075B7A59B
:10064E0075B7F19008D9E090F803F075B7A575B7B6
:10065E00F19008D6E090F804F075B7A575B7F19053
:10066E0008D7E090F805F075B7A575B7F19008D8E2
:10067E00E090F806F075B7A575B7F19008DAE0903E
:10068E00F807F0758F0075D944D2AF2290003FE085
:10069E00B4AB61C2AF75D90475B62275F522758FEC
:1006AE000375B7A575B7F1740090F600F0758F015C
:1006BE00755B00755A00AE5AAF5B7445BE00279F3E
:1006CE00402475B7A575B7F190088F120048E0FC6D
:1006DE0090F600120048ECF0785B740126F6500498
:1006EE0018E436F650D0758F0075F51175B6207575
:1006FE00D944D2AF22C2AF75F52275D904755B000D
:10070E00755A00AE5AAF5B7445BE00229F401F90D3
:10071E00F600120048E493FC90088F120048ECF0AB
:10072E00785B740126F6500418E436F650D575D968
:10073E004475F511D2AF2290003FE0B4AA028003B7
:10074E00020882C2AF75D90475B62275F522758F6F
:10075E000375B7A575B7F1740090F400F075B7A5E1
:10076E0075B7F1740090F200F075B7A575B7F17416
:10077E000090F000F075B7A575B7F1740090EE001B
:10078E00F0758F01755B00755A00AE5AAF5B74FF42
:10079E00C39F74019E402475B7A575B7F19000797B
:1007AE00120048E0FC90F400120048ECF0785B7404
:1007BE000126F6500418E436F650CF755B00755AD4
:1007CE0000AE5AAF5B74FFC39F74019E402475B791
:1007DE00A575B7F1900279120048E0FC90F2001274
:1007EE000048ECF0785B740126F6500418E436F6F7
:1007FE0050CF755B00755A00AE5AAF5B74FFC39F46
:10080E0074019E402475B7A575B7F1900479120056
:10081E0048E0FC90F000120048ECF0785B74012682
:10082E00F6500418E436F650CF755B00755A00AEDC
:10083E005AAF5B74FFC39F74019E402475B7A575B4
:10084E00B7F1900679120048E0FC90EE00120048D5
:10085E00ECF0785B740126F6500418E436F650CFAF
:10086E00758F0075F51175B62075D944D2AF743AEF
:10087E00900779F02290003FE0B4AA0280030209AB
:10088E00C0C2AF75D90475B62275F522758F037582
:10089E00B7A575B7F1740090EC00F075B7A575B7F4
:1008AE00F1740090EA00F075B7A575B7F174009079
:1008BE00E800F075B7A575B7F1740090E600F07515
:1008CE008F01755B00755A00AE5AAF5B74FFC39F04
:1008DE0074019E402475B7A575B7F190007912008A
:1008EE0048E0FC90EC00120048ECF0785B740126B6
:1008FE00F6500418E436F650CF755B00755A00AE0C
:10090E005AAF5B74FFC39F74019E402475B7A575E3
:10091E00B7F1900279120048E0FC90EA001200480C
:10092E00ECF0785B740126F6500418E436F650CFDE
:10093E00755B00755A00AE5AAF5B74FFC39F7401AE
:10094E009E402475B7A575B7F1900479120048E062
:10095E00FC90E800120048ECF0785B740126F6502B
:10096E000418E436F650CF755B00755A00AE5AAFD8
:10097E005B74FFC39F74019E402475B7A575B7F1D4
:10098E00900679120048E0FC90E600120048ECF068
:10099E00785B740126F6500418E436F650CF758F46
:1009AE000075F51175B62075D944D2AF743A90071B
:1009BE0079F022C2AF75D90475F522755B00755AB0
:1009CE0000AE5AAF5B74FFC39F74019E401F90F43C
:1009DE0000120048E493FC900079120048ECF07885
:1009EE005B740126F6500418E436F650D4755B009D
:1009FE00755A00AE5AAF5B74FFC39F74019E401FC1
:100A0E0090F200120048E493FC900279120048EC38
:100A1E00F0785B740126F6500418E436F650D4755F
:100A2E005B00755A00AE5AAF5B74FFC39F74019E94
:100A3E00401F90F000120048E493FC9004791200DD
:100A4E0048ECF0785B740126F6500418E436F65044
:100A5E00D4755B00755A00AE5AAF5B74FFC39F74BA
:100A6E00019E401F90EE00120048E493FC90067920
:100A7E00120048ECF0785B740126F6500418E43648
:100A8E00F650D475F51175D944D2AF74019000C2E9
:100A9E00F0743A900779F09008E87401F022C2AF32
:100AAE0075D90475F522755B00755A00AE5AAF5BA9
:100ABE0074FFC39F74019E401F90EC00120048E427
:100ACE0093FC900079120048ECF0785B740126F6E6
:100ADE00500418E436F650D4755B00755A00AE5AC1
:100AEE00AF5B74FFC39F74019E401F90EA0012001B
:100AFE0048E493FC900279120048ECF0785B7401A4
:100B0E0026F6500418E436F650D4755B00755A007C
:100B1E00AE5AAF5B74FFC39F74019E401F90E800F6
:100B2E00120048E493FC900479120048ECF0785BD4
:100B3E00740126F6500418E436F650D4755B007531
:100B4E005A00AE5AAF5B74FFC39F74019E401F9054
:100B5E00E600120048E493FC900679120048ECF08F
:100B6E00785B740126F6500418E436F650D475F509
:100B7E001175D944D2AF74029000C2F0743A900746
:100B8E0079F074029008E8F02274019000C2F0909F
:100B9E000890E0903C1EF828287380188016A2A3B7
:100BAE00400674029000C2F0800AA2A440067402AD
:040BBE009000C2F0F1
:0C3C1E00020BA8020BAA020BAC020BB8B0
:100BC2009000C2E0B40105A236B34002801AD236C8
:100BD20012464B1209C174019000C2F012039D1219
:100BE2003EB7741B900043F09000C2E0B40206A22C
:100BF20036B3B34002801AC23612464B120AAC74A4
:100C0200029000C2F012039D123EB7741B90004383
:100C1200F022E54F64046006E59964FF60028031CA
:100C2200A22C4004D22C8027E54F600874E6254FA1
:100C3200900043F0E54E600874F0254E900043F0BA
:100C4200E54FB4010280FE754F00754E00C22C8044
:100C520002C22CE54F903C2AF8282873754F00E514
:100C620099B4FF03754E01E599B4FE03754E02E592
:100C720099B4FD03754E03E599B4FC03754E04E582
:100C820099B4FA03754E05E599B4FB06754F011246
:100C9200464BE599B4F906754F0412464BE599B4F3
:100CA200F73312464BC29C74AB90003FF012069A87
:100CB20074AA90003FF09008E8E0B40105120745DD
:100CC200800312088390003FE4F0D29C754F0075B8
:100CD2004E007599F7E599D394E54007E599C394D9
:100CE200F040028016859950754F027E017F00E523
:100CF20050C394E61271288E338F34900887E4F043
:100D0200A3F0E599D394C24007E599C394E6400263
:100D12008028859950754F0374E5C39550F5347555
:100D22003300AE33AF34906A7C1270F7E493F874F8
:100D32000193900887C8F0A3C8F0D2990210A2903C
:100D4200089CE0700AA223B35005A224B34002809B
:100D52005C900887E0FEA3E0FF74FFBE00039F5093
:100D620009EFC39446EE9406402B900887E0FEA359
:100D7200E0FFEFD3946DEE94064009EFC394EEEEDC
:100D820094064011900887E0FEA3E0FFEFD394FFA2
:100D9200EE94064013900887E0FEA3E0FF900079EE
:100DA200120048E599F080038599758011900887B3
:100DB200E0FEA3E0FF900079120048E599F0900868
:100DC20087127136900887E0FEA3E0FFEFB40106B8
:100DD200EEB407028003020E9B900779E0B43C0256
:100DE2008003020E9BA223B35005A224B3400280CB
:100DF20055C29C12039D900086E09008E7F01240D5
:100E020003900165E090089DF0900166E090089ED5
:100E1200F0900167E090089FF074AB90003FF012F1
:100E2200069A74AA90003FF09008E8E0B401051217
:100E3200074580031208839008E8E09000C2F09012
:100E4200003FE4F08048C29C12019C740090089D0F
:100E5200F0740090089EF0740090089FF090008655
:100E6200E09008E7F012400374AB90003FF01206E6
:100E72009A74AA90003FF0120745120883D29C751B
:100E820099FB7464F5097508001205E480FED29C92
:100E9200754F00754E007599FB0210A2900887E00D
:100EA200FEA3E0FFEF4E700685993275310090087F
:100EB20087E0FEA3E0FF74016F4E701BAC31AD32D0
:100EC200AA33AB34ED2BFBEC3AFA8A068B0790007F
:100ED20079120048E599F0900887127136900887D8
:100EE200E0FEA3E0FF74026F4E7021AC31AD3274AC
:100EF200566D4C7006E55064E66002800312464B64
:100F0200124003855099754F00754E000210A29051
:100F12000887E0FEA3E0FF900079120048E599F00F
:100F2200900887127136900887E0FEA3E0FFAC3389
:100F3200AD348F028E038C068D07906AC21270F751
:100F4200E493F9740193FEEAD39EEB99400985502C
:100F520099754F00754E000210A2900887E0FEA31B
:100F6200E0FF900079120048E599F090088712712D
:100F720036900887E0FEA3E0FFEFB40006EEB4016E
:100F82000280030210A2900055E0D394C7400B9058
:100F92000055E0C394C8F551801A900055E0D394EF
:100FA20063400B900055E0C39464F55180069000B5
:100FB20055E0F551E55175F002A4FFAEF08F74EFE4
:100FC200900079127159EFFCE0FDEC90007C1271F7
:100FD20059EDFCE0FDEC2DB5510280030210930F98
:100FE200EF900079127159E574FFE0FCEF90007DFB
:100FF200127159ECFFE0FCEFC39CB5510280030271
:101002001093E57490007B127159E574FFE0FCEFD8
:1010120090007E127159ECFFE0FCEF2CB55172E5A5
:101022007490007F127159E0C395519008D5F0E594
:1010320074900080127159E0C395519008D6F0E582
:1010420074900083127159E0C395519008D7F0E56E
:1010520074900084127159E0C395519008D8F0E55C
:1010620074900085127159E0C395519008D9F0E54A
:1010720074900086127159E0C395519008DAF0120B
:1010820006107599F97464F5097508001205E48073
:10109200FE7599FF7464F5097508001205E480FE77
:0F3C2A00020C5E020D41020E9E020F11020F5C92
:1010A20022E54E903C39F828287302118790088770
:1010B200E0FEA3E0FF900045120048E0F599900899
:1010C20087127136900887E0FEA3E0FF741C6F4E12
:1010D2007003754E00021187856F9902118790087F
:1010E20087E0FEA3E0FF900079120048E0F599EF57
:1010F200B40107EEB40703754E00900887127136EB
:07110200021187900888E04C
:0F3C39000210AC0210AF0210DA0210E002110507
:10110900903CABF82828738553998067856099804E
:1011190062856299805D8566998058856899805352
:10112900856999804E856A998049856B9980449033
:101139000017E0F599803CA22DB340077599FAC2D2
:101149002D8017A222B3400575990F800B9000439B
:10115900E0F599900043E4F0C2228017856C9980EC
:1011690012856799800D856D9980087599FC8003B2
:03117900754E00B0
:103CAB0002111002111502111A02111F0211240226
:103CBB00112902112E021133021138021140021187
:0D3CCB006502116A02116F02117402117975
:0B117C009008871271368003123F12AA
:033C4800021184E2
:1011870022E538255BFFAE5A50010E900079120018
:1011970048E0F539E538255BFFAE5A50010E0FBF21
:1011A70000010E900079120048E0F53A85403CE5D1
:1011B70039B53A058539388041E53AD39539401D27
:1011C700E53AC39539853BF0A4FFAEF0E53C8E04C4
:1011D7008F05FF127118ED2539F538801DE539C3E4
:1011E700953A853BF0A4FFAEF0E53C8E048F05FFF2
:1011F700127118EDF4042539F53822E53AD39539FB
:10120700401DE53AC39539853BF0A4FFAEF0E53CB8
:101217008E048F05FF127118ED2539F538801DE50D
:1012270039C3953A853BF0A4FFAEF0E53C8E048FB9
:1012370005FF127118EDF4042539F5382290007F67
:10124700E0B4017FE56875F00A84FF7E008F38E51A
:101257006875F00A84ADF07C008D3B75400A755ABD
:1012670005755B24E538C394115005121188800673
:101277009005AEE0F538E538C394F05008E53890AE
:101287000067F0800674EF900067F0E56875F00A74
:1012970084FF7E008F38E56875F00A84ADF07C0026
:1012A7008D3B75400A755A05755B5AE538C394112D
:1012B700500512118880069005E4E0F538E538906E
:1012C700003EF02290007FE0B40102800302135930
:1012D700E56875F00A84FF7E008F38E56875F00AC7
:1012E70084ADF07C008D3B75400A755A05755B36F9
:1012F700E538C39411500512118880069005C0E0A7
:10130700F538E538C394F0500585384C8003754CA3
:10131700EFE56875F00A84FF7E008F38E56875F0A1
:101327000A84ADF07C008D3B75400A755A05755BE4
:1013370048E538C39411500512118880069005D2EC
:10134700E0F538E538C394F0500585384D800375CE
:101357004DEF22E56075F00484FF7E008F38E5606D
:1013670075F00484ADF07C008D3B754004755A011F
:10137700755B00E538C3943F5005121188800690CD
:1013870001B8E0F538E538900881F8E4F0E8A3F013
:10139700900042E075F020A4FFAEF09000CAE08E06
:1013A700048F05FF1271188D389000B2E0D3956055
:1013B70050030214659000D6E0D395604010ED907D
:1013C70001B9127159E0F52C752B000214629000D7
:1013D700A1E0D395604043E5389001B9127159E017
:1013E700F539E5389001D9127159E0F53A9000D6F0
:1013F700E0F4042560F53B9000A1E0FE9000D6E004
:10140700F4042EF53CE539B53A05853938800312E1
:10141700120285382C752B008041E5389001D912CE
:101427007159E0F539E5389001F9127159E0F53A4B
:101437009000A1E0F4042560F53B9000B2E0FE9037
:1014470000A1E0F4042EF53CE539B53A05853938B5
:10145700800312120285382C752B0002150C9000A0
:10146700D9E0D395605011E538900239127159E0EF
:10147700F52C752B0002150C9000A2E0D395605057
:1014870043E538900219127159E0F539E5389002B1
:1014970039127159E0F53A9000A2E0F4042560F59D
:1014A7003B9000D9E0FE9000A2E0F4042EF53CE565
:1014B70039B53A05853938800312120285382C75FB
:1014C7002B008041E5389001F9127159E0F539E5B3
:1014D70038900219127159E0F53A9000B2E0F4041D
:1014E7002560F53B9000A2E0FE9000B2E0F4042EE8
:1014F700F53CE539B53A058539388003121202857E
:10150700382C752B00229000EAE0F53D75401175E7
:101517005A02755B00AE52AF53E53D75F00FA4FD5F
:10152700ACF0EDD39FEC9E4021E53D8E048F05FF87
:10153700127118ED75F010A4FFAEF0E56075F011AB
:1015470084FD7C00ED2FF53E800EE56075F011847B
:10155700FF7E00EF24F0F53E853E38E56075F0111B
:1015670084AFF07E008F3B12118885383FAE52AFB3
:10157700539000EAE075F00FA4FDACF0EDD39FECBB
:101587009E4028755A02755B10853E381211888572
:101597003F3985383AAE52AF53E53D8E048F05FF8C
:1015A7001271438D3B853D3C121202E5389008814C
:1015B700F8E4F0E8A3F0752C64752B00229000EA9C
:1015C700E0F53D754011755A02755B00AE52AF5399
:1015D700E53D75F00FA4FDACF0EDD39FEC9E4021E7
:1015E700E53D8E048F05FF127118ED75F010A4FF0D
:1015F700AEF0E56275F01184FD7C00ED2FF53E80BD
:101607000EE56275F01184FF7E00EF24F0F53E854C
:101617003E38E56275F01184AFF07E008F3B121102
:101627008885383FAE52AF539000EAE075F00FA4BB
:10163700FDACF0EDD39FEC9E4028755A02755B1008
:10164700853E38121188853F3985383AAE52AF53F7
:10165700E53D8E048F05FF1271438D3B853D3C129E
:101667001202E538900881F8E4F0E8A3F0E56C6031
:1016770017E56CC394FE50109000DEE0B4020990A9
:1016870000CCE0D3940B5002801F900881E0FEA3AA
:10169700E0FFE56C12712874E78E048F05FF127165
:1016A70018900881ECF0A3EDF09000B4E0B4045F6B
:1016B700E56075F00484FF7E008F38E56075F004FF
:1016C70084ADF07C008D3B754004755A01755B0055
:1016D700E538C3943F500512118880069001B8E0A1
:1016E700F538900881E0FEA3E0FFE5381271287411
:1016F700328E048F05FF127118900881E0FEA3E077
:10170700FFEF2DFDEE3CFC900881ECF0A3EDF075AA
:101717002C64752B002290007FE0B40146E56875C4
:10172700F00A84FF7E008F38E56875F00A84ADF013
:101737007C008D3B75400A755A05755B00E538C31B
:1017470094115005121188800690058AE0F538AE8D
:101757002BAF2CE5382FFF50010E746412716B8E7E
:101767002B8F2C900080E0B40146E56975F00A8460
:10177700FF7E008F38E56975F00A84ADF07C008D37
:101787003B75400A755A05755B6CE538C394115073
:101797000512118880069005F6E0F538AE2BAF2CC0
:1017A700E5382FFF50010E746412716B8E2B8F2C4E
:1017B70090008FE0B40249E56BC3944175F005844E
:1017C700FF7E008F38E56B75F00584ADF07C008DEA
:1017D7003B754005755A06755B00E538C394135091
:1017E70005121188800690068CE0F538AE2BAF2CD9
:1017F700E5382FFF50010E746412716B8E2B8F2CFE
:101807009000D1E0B4020280030218BCE56075F0D5
:101817001584FF7E008F38E56075F01584ADF07C88
:10182700008D3B754015755A03755BF4E538C39415
:101837000B50051211888006900478E0F538E538DA
:1018470075F0FFA4FFAEF09000D2E08E048F05FF85
:10185700127118ED900063F0E56775F078A4FFAE9C
:10186700F074FF8E048F05FF1271188C5A8D5B740C
:10187700028C068D071200398F38AC5AAD5B7404A1
:10188700FF1271438D3B754004755A06755B28E559
:1018970038C3941D500512118880069006BEE0F5E6
:1018A70038AE2BAF2CE5382FFF50010E7464127140
:1018B7006B8E2B8F2C90007EE0B4025DE56275F095
:1018C70064A4FFAEF074081200398E5C8F5D740556
:1018D7008E048F05FF1271188D38AE5CAF5D7405ED
:1018E7008E048F05FF1271438D3B754005755A05B0
:1018F700755BDEE538C39413500512118880069096
:10190700066AE0F538AE2BAF2CE5382FFF50010EF5
:10191700746412716B8E2B8F2C9000C0E0707F90D7
:101927000042E075F00A84FF7E008F38900042E0A5
:1019370075F00A84ADF07C008D3B75400A755A0539
:10194700755BC0E538C3940E500512118880069068
:101957000647E0F538E538900068F09000DFE0B41E
:10196700023C900042E075F00A84FF7E008F3890B9
:101977000042E075F00A84ADF07C008D3B75400AAB
:10198700755A05755BCFE538C3940E50051211885B
:101997008006900656E0F538E538900069F0229009
:1019A7000087E0B401179008DCE0252CFFAE2B5030
:1019B700010E9000DBE012716B8E2B8F2C9000FFD5
:1019C700E0B40114900100E0A852B8000495535008
:1019D70007E560C39561400280139000A9E0252CBC
:1019E700FFAE2B50010E8E2B8F2C021E0D90008701
:1019F700E0B40306A22AB3B3400280509008E6E0A1
:101A070070109008DFE0C39405A852B800069553FC
:101A1700400280109000A9E0252CFFAE2B50010E4C
:101A27008E2B8F2C9008E6E0600D9008DFE0A8521F
:101A3700B800069553400280109000A9E0252CFFBE
:101A4700AE2B50010E8E2B8F2C021E0D900081E0C5
:101A5700B402028003021E0D900084E0602FE56847
:101A6700D39446402890000EE0FEA3E0FF9000BF0D
:101A7700E075F003A4FDACF0EFD39DEE9C400E9013
:101A870000E3E0A852B80005D395535003021E0D9A
:101A97009000B4E0B403028003021C5585625B75B5
:101AA7005A0090008BE0A852B800049553500E904E
:101AB700008CE0A85AB80005D3955B5003021C526E
:101AC700E56275F002A4FFAEF074158E048F05FF72
:101AD7001271188C068D07900609120048FEE0FF68
:101AE700EE900083E0FEEF8E0088F0A4FFAEF07466
:101AF700648E048F05FF1271188C5A8D5B9000421B
:101B0700E075F018A4FFAEF09000CAE08E048F05D0
:101B1700FF1271188C068D07900621120048AE5AE5
:101B2700AF5BE012712874648E048F05FF12711881
:101B37008C5A8D5BE566A85AB80005D3955B5003B0
:101B4700021BC9E566C3955BFFE4955AFE8E5A8F63
:101B57005B7428BE00039F500C755B28755A007490
:101B67000D900043F0AE5AAF5B900084E0127128ED
:101B770074288E048F05FF1271188C5A8D5B90089C
:101B870081E0FEA3E0FF740A8E048F05FF1271182F
:101B97008D068C07AC5AAD5BCFCECF120003740A0B
:101BA7008E048F05FF1271188C5A8D5B900881E0A7
:101BB700FEA3E0FF127173900881EEF0A3EFF0022D
:101BC7001C52E566A85AB80004955B507EAE5AAF22
:101BD7005BE56612716B8E5A8F5B7428BE00039F9C
:101BE700500C755B28755A00740D900043F0AE5A7F
:101BF700AF5B900084E012712874288E048F05FF74
:101C07001271188C5A8D5B900881E0FEA3E0FF7477
:101C17000A8E048F05FF1271188D068C07AC5AAD1A
:101C27005BCFCECF120003740A8E048F05FF1271AB
:101C3700188C5A8D5B900881E0FEA3E0FFEF2DFD25
:101C4700EE3CFC900881ECF0A3EDF0021E0D900035
:101C5700CCE08560F0A4FFAEF0740512712874071C
:101C67001200398E5A8F5B90008BE0A852B800049F
:101C77009553501290008CE075F002A4FDACF0EF84
:101C8700C39DEE9C4003021E0DE56075F00B84FFBB
:101C97007E00900609120048FEE0FFEE900083E008
:101CA700FEEF8E0088F0A4FFAEF074648E048F05FB
:101CB700FF1271188C5A8D5B900042E075F018A4E2
:101CC700FFAEF09000CAE08E048F05FF1271188CEA
:101CD700068D07900621120048AE5AAF5BE01271DD
:101CE7002874648E048F05FF1271188C5A8D5BE57A
:101CF70066A85AB80005D3955B5003021D84E566B4
:101D0700C3955BFFE4955AFE8E5A8F5B7428BE001D
:101D1700039F500C755B28755A00740D900043F0B3
:101D2700AE5AAF5B900084E012712874288E048F3E
:101D370005FF1271188C5A8D5B900881E0FEA3E0B5
:101D4700FF740A8E048F05FF1271188D068C07AC7D
:101D57005AAD5BCFCECF120003740A8E048F05FFF6
:101D67001271188C5A8D5B900881E0FEA3E0FF1278
:101D77007173900881EEF0A3EFF0021E0DE566A8DF
:101D87005AB80004955B507EAE5AAF5BE566127198
:101D97006B8E5A8F5B7428BE00039F500C755B28AF
:101DA700755A00740D900043F0AE5AAF5B900084F3
:101DB700E012712874288E048F05FF1271188C5A4F
:101DC7008D5B900881E0FEA3E0FF740A8E048F0507
:101DD700FF1271188D068C07AC5AAD5BCFCECF12B0
:101DE7000003740A8E048F05FF1271188C5A8D5BDD
:101DF700900881E0FEA3E0FFEF2DFDEE3CFC90088C
:101E070081ECF0A3EDF0229000DFE0B4027BE56007
:101E170075F00884FF7E008F38E56075F00884ADA3
:101E2700F07C008D3B754008755A01755BE0E5381D
:101E3700C3943F50051211888006900278E0F53868
:101E4700E538900883F8E4F0E8A3F0900883E0FE13
:101E5700A3E0FFAC2BAD2C12000374648E048F0536
:101E6700FF127118900883ECF0A3EDF090007CE06E
:101E77008C068D0712712874648E048F05FF12710A
:101E870018900883ECF0A3EDF0900881E0FEA3E042
:101E9700FFAC2BAD2C12000374648E048F05FF1268
:101EA7007118900881ECF0A3EDF090007CE08C06AF
:101EB7008D0712712874648E048F05FF12711890B4
:101EC7000881ECF0A3EDF0A204401DAE52AF5374AD
:101ED70005BE00039F5002D204E562D394CC4008AC
:101EE700D2027411900043F0229000DEE0B40208A1
:101EF7009000CCE0640B60028045900881E0FEA36F
:101F0700E0FFE56C12712874E78E048F05FF1271EC
:101F170018900881ECF0A3EDF09000DFE0B4021F09
:101F2700900883E0FEA3E0FFE56C12712874E78E4A
:101F3700048F05FF127118900883ECF0A3EDF09061
:101F4700009EE05402601B900095E0A852B8001272
:101F5700D39553400DA204B3B35007E562C3949AD7
:101F67004002805FAE35AF36900093E075F002A473
:101F7700FDACF0EF2DFDEE3CFC74022DFD50010C85
:101F8700E562BC003ED39D403A754401A23140331F
:101F9700900094E075F05EA4FDACF07405FF12713B
:101FA700188C5C8D5D124A8F900881E0FEA3E0FFDC
:101FB700900094E02FFF50010E900881EEF0A3EF00
:101FC700F0D231E562A835B8000495365002C23127
:101FD700856236753500E54470030220E69000F10E
:101FE700E0C3954450030220D8900101E0C3940256
:101FF7004003022082E56875F00A84FF7E009005A1
:1020070079120048E0F55B755A00AE5AAF5B900055
:1020170094E012712874648E048F05FF1271188C76
:102027005C8D5D9000F1E004C395448C068D07122A
:1020370071289000F1E08E048F05FF1271188C5CF7
:102047008D5D900881E0FEA3E0FFEF2DFDEE3CFCE7
:10205700900881ECF0A3EDF09000DFE0B4021A9055
:102067000883E0FEA3E0FFAA5CAB5DEF2BFBEE3A33
:10207700FA900883EAF0A3EBF080569000F1E004B1
:10208700C39544854CF0A4FFAEF09000F1E08E04B8
:102097008F05FF1271188C5C8D5D900881E0FEA39F
:1020A700E0FFEF2DFDEE3CFC900881ECF0A3EDF096
:1020B7009000DFE0B4021A900883E0FEA3E0FFAAD5
:1020C7005CAB5DEF2BFBEE3AFA900883EAF0A3EBEB
:1020D700F005449000F1E0C3954450037544009027
:1020E700009EE05401601B900092E0A852B80012D5
:1020F700D39553400DA204B3B35007E560C394CC06
:1021070040028060900090E075F003A4FFAEF0E518
:10211700412FFF50010E74032FFF50010EE560BEE3
:102127000042D39F403E754501A231403790009150
:10213700E075F05EA4FFAEF074058E048F05FF1204
:1021470071188C5C8D5D124A8F900881E0FEA3E0C8
:10215700FF900091E02FFF50010E900881EEF0A351
:10216700EFF0D231E560C395415002C2318560413D
:10217700E54570030222809000F2E0C395455003C5
:10218700022272900101E0C39402400302221CE57F
:102197006875F00A84FF7E00900579120048E0F523
:1021A7005B755A00AE5AAF5B900091E012712874CC
:1021B700648E048F05FF1271188C5C8D5D9000F2A0
:1021C700E004C395458C068D071271289000F2E054
:1021D7008E048F05FF1271188C5C8D5D900881E06D
:1021E700FEA3E0FFEF2DFDEE3CFC900881ECF0A391
:1021F700EDF09000DFE0B4021A900883E0FEA3E060
:10220700FFAA5CAB5DEF2BFBEE3AFA900883EAF08E
:10221700A3EBF080569000F2E004C39545854DF09E
:10222700A4FFAEF09000F2E08E048F05FF12711844
:102237008C5C8D5D900881E0FEA3E0FFEF2DFDEE45
:102247003CFC900881ECF0A3EDF09000DFE0B402D5
:102257001A900883E0FEA3E0FFAA5CAB5DEF2BFBBF
:10226700EE3AFA900883EAF0A3EBF005459000F206
:10227700E0C395455003754500900881E0FEA3E053
:10228700FF9000A3E0BE00039F500D9000A3E090D5
:102297000881F8E4F0E8A3F09000DFE0B4021290C0
:1022A7000883E0FEA3E0FF9000A3E0BE00059F4087
:1022B70002800D9000A3E0900883F8E4F0E8A3F013
:1022C700229000DFE0B401028003022416A204B3C7
:1022D70050030223FD9000AAE0B4017A900881E040
:1022E700FEA3E0FFAC52AD53120003743C8E048F83
:1022F70005FF1271189000BAE0BC00159D401290BE
:102307000881E0FEA3E0FF9000BCE0BE00039F5001
:1023170002D203900881E0FEA3E0FFAC52AD531256
:102327000003743C8E048F05FF1271189000BAE009
:10233700C3940ABC001AD39D4016900881E0FEA3FF
:10234700E0FF9000BCE0C39405BE0004D39F500299
:102357008002C203807A900881E0FEA3E0FFAC52BE
:10236700AD5312000374788E048F05FF1271189015
:1023770000BAE0BC00159D4012900881E0FEA3E082
:10238700FF9000BCE0BE00039F5004D20380419041
:102397000881E0FEA3E0FFAC52AD5312000374784E
:1023A7008E048F05FF1271189000BAE0C3940ABC1F
:1023B700001AD39D4016900881E0FEA3E0FF90002D
:1023C700BCE0C39405BE0004D39F50028002C20341
:1023D700A203B34021900881E0FEA3E0FF9000BB79
:1023E700E012712874648E048F05FF12711890082B
:1023F70081ECF0A3EDF0A203B3400CA235400674C4
:1024070024900043F0D235A2034002C2358002C2B5
:102417000390003EE06006A204B3B3400280199027
:102427000881E0FEA3E0FF90003EE02FFF50010E81
:10243700900881EEF0A3EFF0A201B34006A202B329
:10244700B35009900016E4F0A3F0802D900881E0C6
:10245700FEA3E0FF7400D39F74019E401190088192
:10246700E0F8A3E0900016C8F0A3C8F0800B74FF53
:10247700900016F8E4F0E8A3F09000C1E0C39404DC
:10248700400C9008E3E0C3940240030225709000DB
:10249700AAE0B40147900881E0FEA3E0FF745E1252
:1024A700712874058E048F05FF127118900881EC4E
:1024B700F0A3EDF09000DFE0B4021F900883E0FE88
:1024C700A3E0FF745E12712874058E048F05FF1256
:1024D7007118900883ECF0A3EDF08045900881E037
:1024E700FEA3E0FF745E127128740A8E048F05FF45
:1024F700127118900881ECF0A3EDF09000DFE0B4C2
:10250700021F900883E0FEA3E0FF745E1271287437
:102517000A8E048F05FF127118900883ECF0A3ED63
:10252700F0900881E0FEA3E0FF7402BE000CD39F89
:102537004008752A02752900800A900881E0F5296C
:10254700A3E0F52A900883E0FEA3E0FF7402BE0033
:102557000CD39F4008752E02752D00800A900883C2
:10256700E0F52DA3E0F52E8046900881E0FEA3E07C
:10257700FF7401BE000CD39F4008752A017529001E
:10258700800A900881E0F529A3E0F52A900883E006
:10259700FEA3E0FF7401BE000CD39F4008752E0117
:1025A700752D00800A900883E0F52DA3E0F52E90A5
:1025B7000014E529F0A3E52AF0A238B34009C201C7
:1025C700900016E4F0A3F022900042E09003791205
:1025D7007159E0F542754364900042E0FE9000B502
:1025E700E0D39E4037E56075F00884FF7E008F38A2
:1025F700E56075F00884ADF07C008D3B754008758B
:102607005A03755B96E538C3941F500512118880ED
:102617000690042EE0F5388538438035E56075F07F
:102627000884FF7E008F38E56075F00884ADF07C84
:10263700008D3B754008755A03755BB6E538C39442
:102647001F5005121188800690044EE0F538853832
:1026570043229000EBE0F53D754011755A04755B18
:1026670000AE52AF53E53D75F00FA4FDACF0EDD3CE
:102677009FEC9E4021E53D8E048F05FF127118EDFA
:1026870075F010A4FFAEF0E56075F01184FD7C00D5
:10269700ED2FF53E800EE56075F01184FF7E00EFAB
:1026A70024F0F53E853E38E56075F01184AFF07E85
:1026B700008F3B12118885383FAE52AF539000EB25
:1026C700E075F00FA4FDACF0EDD39FEC9E402875AC
:1026D7005A04755B10853E38121188853F39853855
:1026E7003AAE52AF53E53D8E048F05FF1271438D0D
:1026F7003B853D3C121202853842754364229000A7
:10270700EBE0F53D754011755A04755B00AE52AFAD
:1027170053E53D75F00FA4FDACF0EDD39FEC9E4063
:1027270021E53D8E048F05FF127118ED75F010A499
:10273700FFAEF0E56275F01184FD7C00ED2FF53EEC
:10274700800EE56275F01184FF7E00EF24F0F53E00
:10275700853E38E56275F01184AFF07E008F3B123D
:10276700118885383FAE52AF539000EBE075F00FFC
:10277700A4FDACF0EDD39FEC9E4028755A04755B21
:1027870010853E38121188853F3985383AAE52AFE9
:1027970053E53D8E048F05FF1271438D3B853D3C0C
:1027A7001212028538427543649000E6E0B404795A
:1027B700900042E0FE9000B5E0D39E4037E560759B
:1027C700F00884FF7E008F38E56075F00884ADF06F
:1027D7007C008D3B754008755A03755B96E538C3D9
:1027E700941F5005121188800690042EE0F5388555
:1027F70038438035E56075F00884FF7E008F38E543
:102807006075F00884ADF07C008D3B754008755A03
:1028170003755BB6E538C3941F500512118880060F
:1028270090044EE0F5388538432290007FE0B401EC
:102837003BE56875F00A84FF7E008F38E56875F020
:102847000A84ADF07C008D3B75400A755A05755BAF
:1028570012E538C394115005121188800690059C23
:10286700E0F538E5432538C39464F543900080E0EC
:10287700B4013BE56975F00A84FF7E008F38E5698E
:1028870075F00A84ADF07C008D3B75400A755A05DA
:10289700755B7EE538C39411500512118880069048
:1028A7000608E0F538E5432538C39464F543E54267
:1028B7002543F537900087E0B402109008DBE02548
:1028C70037FE9000DBE0F4042EF5379000DEE0D30E
:1028D70094014040E56CC394E7501D74E7C3956CC1
:1028E700FE9008DDE08E00F5F0E884FF7E008F386B
:1028F700E5372538F537801CE56CC394E7FE90086B
:10290700DDE08E00F5F0E884FF7E008F38E537C301
:102917009538F537A2044006E5422464F537E537D4
:10292700D394644009E537C39464F537800375375A
:10293700009000B7E0C3953750069000B7E0F53731
:1029470022D201900066E0A852B800049553503E89
:10295700900066E0A852B800049553500375370FEE
:10296700900066E004A852B80004955350037537E9
:1029770007900066E02402A852B80004955350025D
:10298700C201900066E060067409900043F0C2300F
:102997007E017F009000BDE01271289000CCE08E90
:1029A700048F05FF127118E560BC000CD39D400829
:1029B700D238740A900043F090007FE0B401099088
:1029C70000BEE0C39568400280159000D0E0A85291
:1029D700B8000495535002C201740B900043F09065
:1029E700007FE0B40107E568C394644002801D904E
:1029F7000116E0600D900116E0A852B80006955345
:102A070040028008C201740B900043F0A20140030A
:102A1700753700C2379000FFE0B40114900100E061
:102A2700A852B8000495535007E560C3956140026A
:102A3700802A9000A8E0D3941D400B9000A8E0C323
:102A4700941EF5378003753700A23440087415903B
:102A57000043F0D237D234D232022B42C232C234D0
:102A6700900087E0B40306A22AB3B34003022B42C7
:102A77009008DFE0C39405A852B8000495535006A8
:102A87009008E6E06002801F9000A8E0D3941D4004
:102A97000B9000A8E0C3941EF537800375370074C8
:102AA7000C900043F0D2379008DFE0A852B800043A
:102AB700955350069008E6E07002801F9000A8E04A
:102AC700D3941D400B9000A8E0C3941EF5378003F4
:102AD700753700740C900043F0D2379008DFE0A8F8
:102AE70052B80004955350319000C6E0B40228D282
:102AF700309008E5E0FE9008E6E0D39E5006900887
:102B0700E6E0700280099008E5E4F0C230800690A4
:102B170008E5E004F08002C2019008DFE02405A880
:102B270052B80004955350139000C6E0B4020A90BF
:102B370008E6E07002D2308002C201A22FB340271C
:102B47009000A8E0D3941D400B9000A8E0C3941E0A
:102B5700F5378003753700A23340067410900043A1
:102B6700F0D233D2378002C23385376D9000A8E0A8
:102B7700D3941D4018900076E02537FE900042E080
:102B870075F01E84FC7F00EE2CF5378029A237B341
:102B97004008900076E0F537801C900078E02537F4
:102BA700FE900076E02EFE900042E075F01E84FC59
:102BB7007F00EE2CF537A238B34005D230756D0093
:102BC70022900042E075F00584FF7E008F38900068
:102BD70042E075F00584ADF07C008D3B75400575CE
:102BE7005A03755BD69000CAE01475F00584FF7E22
:102BF70000E538BE00039F5005121188800BE538A9
:102C070090044F127159E0F538E5389008DEF090DE
:102C170008DEE0FE9000B9E0C39E50089000B9E0DE
:102C27009008DEF09000A8E0D3941D401E9008DEC7
:102C3700E0FE900076E02EFE900042E075F01E84E4
:102C4700FC7F00EE2C9008DEF08031A237B3400AFB
:102C5700900076E09008DEF080229008DEE0FE909B
:102C67000078E02EFE900076E02EFE900042E075A0
:102C7700F01E84FC7F00EE2C9008DEF02290007F8F
:102C8700E0B40136E56875F00A84FF7E00900579A7
:102C9700120048E0F547E547D394644010E547C381
:102CA700946475F00F84FF7E008F4780037547009B
:102CB70090009CE02547F547800690009CE0F5478B
:102CC70022E56875F00A84FF7E00900579120048B6
:102CD700E0C394694007E568D3946440559000E6E3
:102CE700E0C39403502690087BE0FEA3E0FF740442
:102CF700120039E560127128740F8E048F05FF12D8
:102D07007118900879ECF0A3EDF0802490087BE02F
:102D1700FEA3E0FF7404120039E562127128740FF4
:102D27008E048F05FF127118900879ECF0A3EDF06F
:102D3700800F90087BE0F8A3E0900879C8F0A3C85B
:102D4700F0A204401A90087BE0FEA3E0FF74031290
:102D570071287401120039900879EEF0A3EFF09012
:102D6700008FE0B40262E56BC3944175F00584FF00
:102D77007E008F38E56B75F00584ADF07C008D3BE8
:102D8700754005755A06755B14E538C394175005E9
:102D970012118880069006A0E0F538900879E0FEC9
:102DA700A3E0FF740A8E048F05FF127118E5388CB3
:102DB700068D07127128740A8E048F05FF12711889
:102DC700900879ECF0A3EDF0900879E0FEA3E0FF1E
:102DD70090087FE0FCA3E0FDEDD39FEC9E400F90B1
:102DE700087FE0F8A3E0900879C8F0A3C8F022E5CF
:102DF7000875F004A4FFAEF09006BC120048E090FE
:102E07003C4BF8282873804C85537480479000CC3E
:102E1700E08560F0A4FFAEF074081200398F74806B
:102E270033856274802E856874802985697480244F
:102E3700856A74801F856B74801A856C748015850C
:102E470067748010856674800B856D7480069000AA
:042E570017E0F57417
:103C4B00022E0D022E0F022E14022E28022E2D02F2
:103C5B002E32022E37022E3C022E41022E46022E0F
:073C6B004B022E50022E5502
:102E5B00E50875F004A4FFAEF09006BD120048E53E
:102E6B000875F004A4FFAEF0E0FC9006BE1200481B
:102E7B00ECFEE0FFEEC39F4003022F63E50875F005
:102E8B0004A4FFAEF09006BC120048E0B40441E588
:102E9B000875F004A4FFAEF09006BE120048E0C324
:102EAB009574500AE508F50CD39239123DF0E508FC
:102EBB0075F004A4FFAEF09006BD120048E0D39568
:102ECB0074400AE508F50CC39239123DF0022F61EC
:102EDB00E50875F004A4FFAEF09006BD120048E0C3
:102EEB00C395745015E50875F004A4FFAEF0900679
:102EFB00BE120048E0D395745002800AE508F50C29
:102F0B00D39239123DF0E50875F004A4FFAEF090B2
:102F1B0006BD120048E0D395745015E50875F00412
:102F2B00A4FFAEF09006BE120048E0C39574500AA1
:102F3B00E508F50CC39239123DF09006C4E0B401DC
:102F4B00099000D8E0D395625002800A7402F50C08
:102F5B00C39239123DF0806AE50875F004A4FFAE08
:102F6B00F09006BD120048E0D395744015E5087546
:102F7B00F004A4FFAEF09006BE120048E0C39574B7
:102F8B004002800AE508F50CC39239123DF0E508C2
:102F9B0075F004A4FFAEF09006BD120048E0C39597
:102FAB00744015E50875F004A4FFAEF09006BE1250
:102FBB000048E0D39574400AE508F50CD39239121A
:102FCB003DF022AE2FAF3074C9BE000CD39F40082A
:102FDB00782F12717B0230E8753001752F00AE52DD
:102FEB00AF53E547BE000DD39F40099000AEE0D331
:102FFB00954840028023754800E547C39553F57407
:10300B009000B1E0D395464008E5462574F546801F
:10301B00069000B1E0F5468002054890008AE0D3A7
:10302B009562401CE560C395614015AE52AF53E508
:10303B0047BE00039F50099000AFE0D39549400273
:10304B00806E9008E0E0A852B800049553500375C9
:10305B004B009008E0E0A852B8000BD39553400604
:10306B00E5539008E0F0E54B7041E553C39547F508
:10307B0074E574D3940540037574059000B0E0C3F8
:10308B0095465007E574C3954640028009E546C353
:10309B009574F54680069000B0E0F5469000B0E0E0
:1030AB00D3954640069000B0E0F546754900800286
:1030BB000549E54B701690008AE0C39562500DE50B
:1030CB00472405A852B8000695534002800F900084
:1030DB009DE0F546754B0174789008E0F022AE2F19
:1030EB00AF3074E9D39F74039E4008782F12717B25
:1030FB0002328F753001752F00754632A22B402A94
:10310B0075461990009DE075F002A4FFAEF0E548FE
:10311B00BE0006D39F4002D22B0548754B03747833
:10312B009008E0F0754A00023276AE52AF53E54795
:10313B006F4E7003023276E547BE000DD39F4009F8
:10314B009000AEE0D395484002800F754800E54BE8
:10315B00C394035003754619800DE547C39553F58A
:10316B0074E5482574F54890008AE0D39562400ECB
:10317B009008E0E0A852B80007D395534002800CAA
:10318B00054A90009DE0B54A03754B00E54BB4032F
:10319B0006A204B3B34002800A054AE54AB43C03D5
:1031AB00754B02E54BB402299008E0E0A852B80039
:1031BB000ED395534009E5539008E0F0754A009003
:1031CB00008AE0C395625009754A0074789008E054
:1031DB00F0E54B705A90008AE0D39562401CE56095
:1031EB00C395614015AE52AF53E547BE00039F50E8
:1031FB00099000AFE0D395494002800875490075EE
:10320B00464B8028E553C39547F574E574D3940575
:10321B00400375740590008AE0D395624008E54938
:10322B002574F5498006E5492406F549754A00E5FC
:10323B004B701690008AE0C39562500DE54724054C
:10324B00A852B80006955340028003754B01E54B1D
:10325B00B40118754619054A90009DE0B54A0675EC
:10326B004B02754A0074789008E0F0A202B3400359
:10327B00754632E54675F00AA4FFAEF0900885EE70
:10328B00F0A3EFF022E570903C72F8282873023C13
:10329B000B900082E070030235BA9000B8E0B401E5
:1032AB00028003023450900040E0655F6009E553F3
:1032BB004552600302344D7E017F00E5BE1271283A
:1032CB00E5BD2FFF50010E8E5A8F5B9000B6E0B418
:1032DB00461B740E127128900065E08E048F05FF5B
:1032EB00127118900889ECF0A3EDF0801DAE5AAF67
:1032FB005B7410127128900065E08E048F05FF122D
:10330B007118900889ECF0A3EDF0E56C600FE56C9B
:10331B00C394FE50089000DEE0640260028064906B
:10332B0000CCE0B40B1F900889E0FEA3E0FF74E72C
:10333B00127128E56C8E048F05FF127118900889A5
:10334B00ECF0A3EDF09000CCE0D3940B4008900090
:10335B00B4E064046002802B900889E0FEA3E0FFD8
:10336B0090088DE0FCA3E0FDEFD39DEE9C400D1289
:10337B007173900889EEF0A3EFF08007900889E451
:10338B00F0A3F0900889E0FEA3E0FFEFD39400EEEA
:10339B0094014008D2387426900043F0A238B3B39E
:1033AB00502C7E057F009000CCE08E048F05FF1221
:1033BB007118900889E0FEA3E0FFEFC39DEE9C40DF
:1033CB000FAC52AD53740FBC0004D39D500280025E
:1033DB00C238900082E0B4022790088BE0FEA3E095
:1033EB00FF900889E0FCA3E0FDEF2DFDEE3CFC74A3
:1033FB00018C068D07120039900889EEF0A3EFF0CF
:10340B00900889E0FEA3E0FF90088BE0FCA3E0FDB1
:10341B00EDD39FEC9E4004D22E8002B22E900889F1
:10342B00E0F8A3E090088BC8F0A3C8F09000B4E0DC
:10343B0064016006A22EB3B34002800690088AE0B6
:10344B00F5600235B8D22E7E017F00E5BE127128E1
:10345B00E5BD2FFF50010E8E5A8F5B9000B6E0B486
:10346B00461B740E127128900065E08E048F05FFC9
:10347B00127118900889ECF0A3EDF0801DAE5AAFD5
:10348B005B7410127128900065E08E048F05FF129B
:10349B007118900889ECF0A3EDF0E56C600FE56C0A
:1034AB00C394FE50089000DEE064026002806490DA
:1034BB0000CCE0B40B1F900889E0FEA3E0FF74E79B
:1034CB00127128E56C8E048F05FF12711890088914
:1034DB00ECF0A3EDF09000CCE0D3940B40089000FF
:1034EB00B4E064046002802B900889E0FEA3E0FF47
:1034FB0090088DE0FCA3E0FDEFD39DEE9C400D12F8
:10350B007173900889EEF0A3EFF08007900889E4BF
:10351B00F0A3F0900889E0FEA3E0FFEFD39400EE58
:10352B0094014008D2387426900043F0A238B3B30C
:10353B00502C7E057F009000CCE08E048F05FF128F
:10354B007118900889E0FEA3E0FFEFC39DEE9C404D
:10355B000FAC52AD53740FBC0004D39D50028002CC
:10356B00C238900082E0B4022790088BE0FEA3E003
:10357B00FF900889E0FCA3E0FDEF2DFDEE3CFC7411
:10358B00018C068D07120039900889EEF0A3EFF03D
:10359B00900889E0F8A3E090088BC8F0A3C8F090DE
:1035AB0000B4E06401600690088AE0F56080037562
:1035BB00600090007EE0700675700302329075BB60
:1035CB0018023C0B023C0B90007EE0700302374369
:1035DB007E017F00E5BE127128E5BD2FFF50010E65
:1035EB008E5A8F5B9000C4E0B4010F7E0F7FFFAC4F
:1035FB005AAD5B1271738E5A8F5B9000E9E0B40287
:10360B0045AE5AAF5B900020E0FCA3E0FDEDD39FED
:10361B00EC9E400A900020E55AF0A3E55BF0AE5A11
:10362B00AF5B900022E0FCA3E0FDEFD39DEE9C404E
:10363B000A900022E55AF0A3E55BF0AE5AAF5B743B
:10364B00041200398F629000E9E0704CAE5AAF5B08
:10365B00900020E0FCA3E0FDEFD39DEE9C4009120F
:10366B0071738E5A8F5B8006755B00755A00AE5A6C
:10367B00AF5B74101271289000E8E08E048F05FF89
:10368B001271188C5A8D5B74FFBC0009D39D4005D9
:10369B00855B6280037562FE9000B4E0B40102802A
:1036AB0003023741A204B3B3500E900088E0A85236
:1036BB00B80005D39553500280719000C5E0856228
:1036CB00F0A4FFAEF074648E048F05FF1271188C9A
:1036DB005A8D5BE56C6016E56CC394FE500F900041
:1036EB00DEE0B402089000CCE0640B60028017AE01
:1036FB005AAF5B74E7127128E56C8E048F05FF12CD
:10370B0071188C5A8D5BAE5AAF5B900889E0FCA3A5
:10371B00E0FDEDD39FEC9E4005855B60800BA22EF8
:10372B00B3400690088AE0F560800BA22EB34006EA
:10373B0090088AE0F5608003756200900081E0706C
:10374B000675700502329075BB19023C0B023C0BDF
:10375B00900081E070030237FBE55FD3955E400379
:10376B000237F990001EE0FEA3E0FFE56612716BD5
:10377B0090001EEEF0A3EFF07E017F00E5BE12710C
:10378B0028E5BD2FFF50010E8E5A8F5B9000EEE0A7
:10379B007013740A12712874518E048F05FF127105
:1037AB00188D668019AE5AAF5B740A1271288F049C
:1037BB008E057E017F95CDCCCD1270168F66E5669A
:1037CB00D39464400375666490001EE0FEA3E0FF93
:1037DB00E5662FFF50010E90001EEEF0A3EFF09068
:1037EB000085E0048E048F05FF1271188D6680032F
:1037FB007566329000D1E0700675700702329075D5
:10380B00BB13023C0B023C0B9000D1E0604A7E01E3
:10381B007F00E5BE127128E5BD2FFF50010E8E5AB9
:10382B008F5B74041200398F679000D3E08567F0CB
:10383B00A4FDACF07464FF1271188D679000D2E098
:10384B008567F0A4FFAEF074FF8E048F05FF127135
:10385B0018ED900064F0800375670090007FE070B6
:10386B000675700902329075BB17023C0B023C0BBC
:10387B0090007FE0B40102800302390F7E017F00CC
:10388B00E5BE127128E5BD2FFF50010E8E5A8F5BDE
:10389B009008E1E060199008E1E014906B081200C9
:1038AB008CE493FC740193FDEDC39FEC9E4002806E
:1038BB00069008E1E014F09008E1E0C394B3501DCA
:1038CB00AE5AAF5B9008E1E004906B0812008CE4F9
:1038DB0093FC740193FDEFC39DEE9C400280069018
:1038EB0008E1E004F09008E1E0FE9000A5E08E0016
:1038FB0088F0A4FFAEF074648E048F05FF1271186C
:10390B008D688003756800900080E0700675700B01
:10391B0002329075BB16023C0B023C0B900080E010
:10392B00B4010280030239BB7E017F00E5BE127138
:10393B0028E5BD2FFF50010E8E5A8F5B9008E2E0F9
:10394B0060199008E2E014906C7212008CE493FC06
:10395B00740193FDEDC39FEC9E400280069008E23C
:10396B00E014F09008E2E0C394B3501DAE5AAF5B85
:10397B009008E2E004906C7212008CE493FC7401EA
:10398B0093FDEFC39DEE9C400280069008E2E0049D
:10399B00F09008E2E0FE9000ABE08E0088F0A4FF10
:1039AB00AEF074648E048F05FF1271188D6980035D
:1039BB0075690075BB1F023C0B023C0B7E017F003F
:1039CB00E5BE127128E5BD2FFF50010E8E5A8F5B9D
:1039DB00740912712874E68E048F05FF1271188D0D
:1039EB006B900087E0700675700F02329075BB15F7
:1039FB00023C0B023C0B900087E07003023B527EB3
:103A0B00017F00E5BE127128E5BD2FFF50010E8E20
:103A1B005A8F5B74041200398F6A900087E0B401EF
:103A2B00159000DBE0856AF0A4FFAEF0740712007E
:103A3B0039EF9008DCF0900087E0B402159000DBC2
:103A4B00E0856AF0A4FFAEF07407120039EF90081E
:103A5B00DBF0900087E0B403028003023B3590005B
:103A6B00C8E07052E56AC39419500FD22A9000A790
:103A7B00E09008DFF09008E4E4F0E56AD39464404A
:103A8B0004A22A4002802D9008E4E004F09008E4A0
:103A9B00E0FE90011AE0B5060B9008DFE004F09011
:103AAB0008E4E4F09008DFE06496600690011AE009
:103ABB007002C22A80639000A7E070349000DBE0B4
:103ACB00856AF0A4FFAEF074FF8E048F05FF1271B0
:103ADB0018ED9008DFF0AE52AF53741EBE0006D344
:103AEB009F4002D22AE562D394E54002C22A802984
:103AFB00E56AC3940A500DAE52AF53741EBE000458
:103B0B00D39F50028002D22AE562D394E54002C2D1
:103B1B002A9000A7E09008DFF09008DFE0C394053F
:103B2B00500674059008DFF0C22F900087E0B404B4
:103B3B0014E56AC394195002D22FE56AD39432402C
:103B4B0002C22FC22A8003756A009000DEE0700665
:103B5B0075701102329075BB14023C0B023C0B903A
:103B6B0000DEE07003023BF87E017F00E5BE1271C0
:103B7B0028E5BD2FFF50010E8E5A8F5B900103E09D
:103B8B007025EFD39421EE940E4005756CFF8015D4
:103B9B00AE5AAF5B741012712874E38E048F05FF5D
:103BAB001271188D6C8027AE5AAF5BEFD39449EE30
:103BBB0094064005756CFF8015AE5AAF5B741012FE
:103BCB00712874638E048F05FF1271188D6CE56C70
:103BDB0075F00BA4FFAEF09000CCE08E048F05FFC8
:103BEB0012711890088DECF0A3EDF08003756C004A
:103BFB00900082E0600575BB1A800375BB188000CE
:103C720002329902329C0235CF0235D20237580203
:103C8200375B02381002381302387802387B023967
:103C9200240239270239C40239C70239FE023A0125
:093CA200023B67023B6A023C0B85
:103C0B00E57075F00284AFF07E00EF4E7002D2ECDF
:033C1B000570220F
:097159002582F582500205832213
:0F008C0025E050020583258250020583F582226C
:1070F700EF2F500205832582F582E5833E2EF58327
:017107002265
:10716B00CFC39FFF50011E22C3EF9DFFEE9CFE225B
:08717B000806B6000218062206
:0D713600A3E004F0700612714FE004F02297
:0E003900048007C3CE13CECF13CFD5E0F6223E
:10701600BC000FBE0008ED8FF084FFADF022E4FE49
:10702600FF22BE000DEF60FE54F0606F20E7030202
:1070360070CCEAC0E0EBC0E078017A0075F001EEB2
:1070460020E710EF25E0FFEE33FE0AC5F023C5F07A
:1070560030E7F0EA5407F9096A7A007B0060010814
:10706600C3EC9E40167004ED9F4010ED9FFDEC9E14
:10707600FCE5F0CA4ACA03F5F08005E5F003F5F031
:10708600C3EE13FEEF13FFD9D77908CACBCAD8D0FF
:10709600EAFEEBFFD0E0FBD0E0FA22EC8FF084FCB6
:1070A600ED54F045F0C48FF084FEEDC454F045F085
:1070B600C48FF084FDEEC4FE54F02DFFEE540F3C59
:1070C600FEADF07C0022790078008FF0EC7E08207F
:1070D600E70DC3CD33CD33C933C9C833C8DEF08419
:1070E60049F9E5F08FF0BE00E6FD7C00E9FFE8FE19
:0170F6002277
:0E712800F88FF0A4FFE5F0CE88F0A42EFE2232
:10000300EF8DF0A4F9A8F0EF8CF0A428F8EE8DF0B2
:06001300A428FEE9FF2213
:10710800600D782B027112007830D8FED5E0F82295
:10711800EEC0E07E00127016EFFDEEFCD0E0FE221D
:0C714300EEC0E07E00127016D0E0FE22CC
:03001B0002001EC2
:0300530002005652
:03009B00020071EF
:0300000002716228
:0971620075817675D000024BF82E
:0B004800E5822FF582E5833EF5832260
:0A714F000582D58202158315822205
:10001E00C0E0C0F0C083C082C0D075D000124B6269
:0B002E00D0D0D082D083D0F0D0E032E0
:10005600C0E0C0F0C083C082C0D075D000124B652E
:10006600D0D0D082D083D0F0D0E032C0E0C0F0C093
:1000760083C082C0D075D000124BBAD0D0D082D007
:0600860083D0F0D0E0324F
:00000001FF
